:062000003FEF10F0534712
:10200800FACF40F0FBCF41F0E9CF42F0EACF43F0FE
:10201800E1CF44F0E2CF45F0D9CF46F0DACF47F030
:10202800F3CF48F0F4CF49F0F6CF4AF0F7CF4BF0B2
:10203800F8CF4CF0F5CF4DF0DEEC92F04DC0F5FF47
:102048004CC0F8FF4BC0F7FF4AC0F6FF49C0F4FF89
:1020580048C0F3FF47C0DAFF46C0D9FF45C0E2FFDA
:1020680044C0E1FF43C0EAFF42C0E9FF41C0FBFFB3
:0A20780040C0FAFF1100B5EFA2F01E
:10F4E600000D0102030405060708090A1624000E8A
:10F4F6000E0E0E0E0E0E0E0B2F54180E0E0E414251
:10F506000E0E0E235F550C0E0E0E4D4E0E0E0E17E2
:10F516005E5619252627282B2C2D2E225D57303195
:10F526003233343738393A3B5C583C3D3E3F4043F2
:10F53600444546475B5948494A4B4C4F50515253F4
:10F546005A2F3B3C3D3E3F40414243442E353A0014
:10F55600000000000000004531301E0000000000E1
:10F56600000000272D2A1F20212200002324252603
:10F5760034141A09130A00000D0F181C330415164B
:10F58600170729650B11080C121D1B0619052B28D8
:10F596000E10363738E0E3F0E12CE2E62CE5F1E731
:10F5A600E42F3B3C3D3E3F404142434431353A0027
:10F5B60000000000000000452E301E000000000084
:10F5C6000000002738391F20212200002324252689
:10F5D6002D343637131C0000090A06150F041208CD
:10F5E600180C2965070B17111633140D0E1B2B2843
:10F5F60005101A191DE0E3F0E12AE2E62CE5F1E731
:10F60600E4303B3C3D3E3F40414243442E893A0074
:10F6160000000000000000452F321E000000000020
:10F62600000000272D391F20212200002324252633
:10F6360034141A08151700001C180C1213041607A8
:10F64600090A29650B0D0E0F331D1B0619052B28FC
:10F656001110363738E0E3F0E12AE2E62CE5F1E76F
:10F66600E4303B3C3D3E3F40414243442D893A0015
:10F6760000000000000000452F321E0000000000C0
:10F6860000000027342E1F202122000023242526D7
:10F696002A141A08151700001C180C121304160752
:10F6A600090A29650B0D0E0F331D1B0619052B289C
:10F6B6001110363738E0E3F0E158E2E62CE5F1E7E1
:10F6C600E42F3B3C3D3E3F40414243442E353A0009
:10F6D600000000000000004531301E000000000060
:10F6E600000000272D391F20212200002324252673
:10F6F60034141A08151700001C180C1213041607E8
:10F70600090A29650B0D0E0F331D1B0619052B283B
:10F716001110363738E0E3F0E12AE2E62CE5F1E7AE
:10F72600E4000102030405060708090A0B030102A7
:10F7360000040506070B090A080001020403050672
:10F746000807090A0B030102040005060B07090A4C
:10F75600080000005500FB00675400005F6061561A
:10F76600005C5D5E5700595A5B280062006300002A
:10F77600040C1808121CFBFF2FFFEAFD0A1D0705E3
:10F7860014FEE02F003B00003C00003D00003E0060
:10F79600003F00004000004100004200007F0000E2
:10F7A6008100004800004900003A00000000000007
:10F7B6000000000000000000000000000000000043
:10F7C60000000000800000470000E0E11DE01E0090
:10F7D6000000000000000000000000000000000023
:10F7E6000000000000000000E027004600004C007A
:10F7F60000E01F00E02000E02100E0220000000001
:10F80600000000E02300E02400E02500E02600538D
:10F816000000E01C00E01A004B0000E01500E017B5
:10F8260000000000000000E04A00E0500052000026
:10F83600E04F00E04D00E00400E016004E0000E05E
:10F846000900E00A002900003900004A00005000C3
:10F85600005100004F00004D0000E01D00E01B00BD
:10F86600E00600E01900E005002B0000280000E09B
:10F876001100E15000E15100E14F00E14D000000B0
:10F8860000000000000000000000E02A0000000068
:10F89600000000E02C000000000000000000000056
:10F8A6000000000000000000000000000000000052
:10F8B6000000000000000000000000000000000042
:10F8C6000000000000000000000000000000000032
:10F8D6000000B69AB5B4B300002A31383F46040397
:10F8E6000201050000070E151C23AE6993A4B200A1
:10F8F600004D545BCD6200000000000000000000D7
:10F9060000000000000000000000000000000000F1
:10F9160000000000000000000000000000000000E1
:10F92600000000000000ACA9A6A2B00000307A3E9C
:10F93600C84CABA8A5A1AF00000D141B2229ADAA87
:10F94600A7A3B10000535A61CE68E600000000008C
:10F956000000000000CA00000000000000000000D7
:10F966000000E700000000000000000000CD0000DD
:10F9760000000000000000000000CE08160C0F007A
:10F986000039170A18CD0310190B120000241A09A2
:10F9960002C8CE2511262700002E132028ECE600EB
:10F9A600000000000000000000CA00000000000087
:10F9B600000000000000E7CC00000000000000008E
:10F9C60000CD00EDF1E6E70000EAEB0000006A0476
:10F9D6003A7F3C0000475D505E4844011D812F0080
:10F9E6000063604F4BC86CC93D326B000049594AF1
:10F9F60067ECE800000000000000000000CB0000FB
:10FA060000000000000000000000E9CC000000003B
:10FA16000000000000CD00EDF1E6E70000EAEB0093
:10FA26000000CE4E5C52550000361E3B2B6D96569E
:10FA36005F515800002C0521837ACE645765660015
:10FA4600001F342D406ED3000000000000000000AF
:10FA56000000000000000000000000000000D4D7F5
:10FA6600000000000000000000DE000000000000B2
:10FA76000000000000DD00000000000000000000A3
:10FA860000D100000000000000000000000000009F
:10FA9600DB0000000000000000E0D30000000000D2
:10FAA6000000000000000000000000000000000050
:10FAB6000000D400000000000000000000DE00008E
:10FAC600000000000000000000DF000000B300009E
:10FAD6000000000000D2000046D6D5000000D9D8AC
:10FAE600DC000000000000000000DA000000E60074
:10FAF6000000000000000000000000000000000000
:10FB0600000000000000E700000000000000000008
:10FB16000000000000000000000000000000393B6B
:10FB26000C2483000009210A013C161A08192F002B
:10FB36000044020310C82B3A1E0F1D00001118CDF9
:10FB4600CE7AE60000000000000000000000EE0093
:10FB560000000000000000000000E70000000000B8
:10FB6600000000000000000000000000000000008F
:10FB760000002513EC7F2800004F5150CC8E1F202B
:10FB86008136260000CA5D9656906D6E12342700A7
:10FB960000575EEFF086E80000000000000000005D
:10FBA6000000000000000000000000000000E90066
:10FBB600000000000000000000000000000000003F
:10FBC60000000000000064595263670000040B2E19
:10FBD6002D3D5C604E5F6500000517C92C327174BF
:10FBE6005855660000406B6ACB6CE60000000000CA
:10FBF60000000000000000000000000000000000FF
:10FC06000000E700000000000000000000170000F0
:10FC16000000000000000000001D130B12198300F5
:10FC26000018C821443A2408101A1600000A0302D4
:10FC3600CA09110C1E0F0100007A3BCDCE3CE8002C
:10FC460000000000000000000000000000000000AE
:10FC5600000000000000E9000000000000000000B5
:10FC660000E60000000000000000000000E76ACB8C
:10FC760028262E000025042C321F6B2739813600DA
:10FC8600002B052F40346C6D6E207F00002D3DEC5F
:10FC9600C9CC041111040E18041718040C000C1119
:10FCA600110C0E180C1718181111180E1818171811
:10FCB600081111080E0C081718080C001211111261
:10FCC6000E181217181218000600000900000D0081
:10FCD6000014000005010906A101050719E029E73E
:10FCE60015002501750195088102950175088103A6
:10FCF60095057501050819012905910295017503F8
:10FD0600910395067508150026FF000507190029B9
:10FD1600FF8100C0062800000016280000001B0610
:10FD26002800001B16280000060D280000160D28C6
:10FD360000001B060D28001B160D2800060D0428C2
:10FD460000160D0428001B060D04281B160D04289A
:10FD560011112D00F300F400E13836003700E136CA
:10FD6600E1372F003000E130E13234002E002D0063
:10FD76001E0038003200E1278700E136E137E1381E
:10FD86008900E11E130628000010040628001E271D
:10FD96002104281E272105281E272628001E27267F
:10FDA60004281E27260528042D161328162D16139B
:10FDB60028062D16132800000E0016001700110045
:10FDC6000B0010001C0015001A0013000A001D008D
:10FDD600070005001B001B0E1B171B1C1B1A1A1CF9
:10FDE60019000F002A0345007300720069006C00B9
:10FDF6006C00650020004E006500770020004B0077
:10FE06006500790062006F006100720064000902FB
:10FE16002900010100A032090400000203010100CB
:10FE26000921110100012240000705810308000194
:10FE3600070501030800012F0000300000E12F0034
:10FE4600E13000E2E126E2E1273800003800003820
:10FE56003838360000370000E135002F000030004A
:10FE6600002F00003000002F000030000038000096
:10FE7600380000383838360000370000E135002FEA
:10FE860000003000001D2F001D30002F0000300044
:10FE9600001D38003800001D37003600003700000E
:10FEA600E13500151210042800110C06122800175F
:10FEB600151211280016170C060E281B23272721BA
:10FEC6002810171C1308282F00003000002F0000F0
:10FED6003000002F000030000038000038000038E5
:10FEE6003838360000370000E135000612131C15BD
:10FEF6000C0A0B172C1F271E202D1F271F272C0827
:10FF060016150C0F0F082C0C11063728000F2800A9
:10FF16000006280000152800000F2D1128062D06C2
:10FF260028152D1628120909281A03450073007290
:10FF36000069006C006C006500200049006E0063DB
:10FF4600002E00181628000018162D072818162D42
:10FF560006280D132800000D132D11280727280049
:10FF6600071E1F28071F21280720232807212528C9
:10FF760010162800000417120E280A12120A280466
:10FF860013130F281201000200000008D80450F5D0
:10FF96000100010200010816150C0F0F082C110CA8
:10FFA60016160828008B00008A000088000035001D
:10FFB6000012090928121128000F0807280000005E
:10FFC6000002040000150819372C00190815372CF3
:10FFD60000091F2C0009202C0009212C0009222CC5
:10FFE6000009232C0009242C0009252C0009262CA5
:0AFFF600000E16170B0403090400A7
:020000040001F9
:1000000083C0D9FF84C0DAFFDF5000019C6F020E6D
:100010000001A46F010E0001916F83C0D9FF84C05D
:10002000DAFFDF50DD0B0001966F87C0D9FF88C073
:10003000DAFF96C0DFFF020E0001956FF8D20001D3
:1000400095510001686F696B68BF6907000E000178
:100050006B6F010E6A6F32ECABF00001685100016A
:100060008325D96E0001695100018421DA6EDF50C9
:100070000001A16FA1C060F00001616B000E0001E2
:10008000636F0C0E626F5DEC9FF000016051000128
:10009000A06FA1C060F00001616B000E0001636FF2
:1000A0000C0E626FACECA1F0000160510001976F83
:1000B0000001A15160ECA2F00001A36F0001A35167
:1000C0000001D8B42AD00001A451010DF350000161
:1000D0008725D96EF45000018821DA6EA3C0DFFFB6
:1000E0000001A42BF70E0001606F010E0001616F8B
:1000F000000E0001636F000E626F000E0001656F5D
:10010000030E646F4EECABF01CD183C0D9FF84C0EA
:10011000DAFFDF500001966F87D2000E0001926F68
:1001200000019C51220B220AD8A410D00101CDA3BA
:1001300003D000019C930AD085C0D9FF86C0DAFFA6
:100140000001DFAA03D000019C9B00D0060E000135
:10015000A06504D0000E0001A26F36D000019CA360
:1001600008D00001A0510C0D8BC08FF08CC090F016
:1001700012D000019CAB08D00001A0510C0D8DC025
:100180008FF08EC090F007D00001A0510C0D89C0F7
:100190008FF08AC090F0F35000018F27F4500001D7
:1001A000902300019751010DF35000018F27F45067
:1001B000000190238FC0F6FF90C0F7FF000EF86E8D
:1001C0000800F5CFA2F000D00001A2510001D8B480
:1001D00045D0D00E0001A26505D0E00E0001A26559
:1001E0003DD000D0010E0001926F020E0001986F09
:1001F00000019851800A780FD8B030D001D02ED0AD
:10020000000198510001686F696B68BF6907000EB3
:1002100000016B6F010E6A6F32ECABF000016851A8
:1002200000018525D96E0001695100018621DA6E31
:100230000001A151DE18D8A40DD00E0E0001A16F4F
:10024000010E0001A06F020E0001976F000E000169
:10025000A26F04D00001982BCBD700D00001A2518F
:100260000001D8B40BD09D0E0001786F000E000184
:10027000796F0001A251C8EC89F000D00001A251B1
:100280000001D8B405D000019D510001D8A462D06E
:100290000001A151CFEC98F00001A36F0001A35120
:1002A0000001D8B4C1D183C0D9FF84C0DAFFDF50C8
:1002B0000001686F020E000185250001606F000ECD
:1002C000000186210001616FA3C062F00001636B31
:1002D000000E0001656F060E646FA7ECA6F000012A
:1002E000605100016111D8A402D0010E01D0000EAE
:1002F0000001696F0001A35151ECA5F00001A36F4B
:100300000001A451010DF35000018725D96EF4506E
:1003100000018821DA6EA3C0DFFF0001A42BF70ED5
:100320000001606F010E0001616F000E0001636F3C
:10033000000E626F000E0001656F030E646F4EECDD
:10034000ABF083C0D9FF84C0DAFFDF500101CD6F6D
:10035000DCD66AD1000192510001D8B460D0000E01
:100360000001996F48D0000E00019A6F2DD0000156
:100370009A51010D9D0EF324D96E000EF420DA6E11
:1003800000019951010DFA0EF324E16E010EF420E3
:10039000E26EDE50E618D8A414D0FA0E0001606FA9
:1003A000010E0001616F000E0001636F000E626FAD
:1003B000000E0001656F030E646F4EECABF0020E91
:1003C000120000019A2B00D000019A51800A7D0F83
:1003D000D8B00ED000019A51010D9D0EF324D96EB4
:1003E000000EF420DA6EDF50D8B402D0C0D700D0AF
:1003F0000001992B00D000019951800A7D0FD8B0DF
:100400000ED000019951010DFA0EF324D96E010EA0
:10041000F420DA6EDF50D8B402D0A5D700D0030E96
:100420000001916F000E00019B6FCCD000019B5129
:10043000010D9D0EF324D96E000EF420DA6EDF500C
:100440000001A36FADD00101F751D8B4B8D0F70EB9
:100450000001606FFF0E0001616FF7C162F00001E3
:10046000636B000E0001656F040E646FA7ECA6F0CD
:1004700060C093F061C094F00001935100019411A9
:10048000D8B49DD0060E0001A46199D00001A451FA
:10049000010DF35000018725D96EF4500001882129
:1004A000DA6E2A0EDF6E0001A42BF70E00018F6FAB
:1004B000FF0E0001906F00018F1F901F8F4B902B3C
:1004C0000001935100018F270001945100019023F6
:1004D000820E00018F25F66EF70E9021F76EF86AF6
:1004E000000EF8220001A451010DF35000018725F0
:1004F000D96EF45000018821DA6E0800F5CFDFFFD5
:1005000034D00001A451010DF35000018725D96EAC
:10051000F45000018821DA6EF8C1DFFF29D04FD0F6
:100520000B0E0101F719D8A44AD0060E0001A461F0
:1005300046D00001A451010DF35000018725D96E6A
:10054000F45000018821DA6E2A0EDF6E0001A42B20
:100550000001A451010DF35000018725D96EF4501C
:1005600000018821DA6E130EDF6E0001A42BC9D7BB
:100570000001A42B24D00001968321D00001968B8A
:100580001ED00001A451010DF35000018725D96E42
:10059000F45000018821DA6EA3C0DFFFE9D70FD045
:1005A0000001A351E10AD8B4E6D7040AD8B4E6D7CB
:1005B000160AD8B448D7070AD8B4B2D7E2D7000190
:1005C0009B2B00D000019B51800A7D0FD8B011D029
:1005D00000019B51010D9D0EF324D96E000EF420F5
:1005E000DA6EDF50D8B405D0070E0001A4651ED71F
:1005F00000D0F70E00016E6F010E00016F6F9D0EAF
:100600000001706F000E0001716F000E0001736F2A
:10061000030E726F10ECA7F083C0D9FF84C0DAFF1D
:10062000DF500101CD6F00D00001952B00D00001FB
:100630009551800A780FD8B005D0070E0001A46547
:10064000FED400D0020E0001A4651AD0FA0E0001FB
:100650006E6F010E00016F6FF70E0001706F010EDB
:100660000001716F000E0001736F030E726F10ECCA
:10067000A7F087C0D9FF88C0DAFF96C0DFFF1DD082
:10068000FA0E0001606F010E0001616F000E0001A3
:10069000636F000E626F000E0001656F030E646FE2
:1006A0004EECABF083C0D9FF84C0DAFF87C0E1FF16
:1006B00088C0E2FFDFCFE7FF00D0000191511200B8
:1006C0001200ABC060F0ACC061F0ADC062F0AEC073
:1006D00063F0000E0001656F080E646F8EECA4F0ED
:1006E0000001605100016111D8A402D0000E120077
:1006F000AFC060F0B0C061F0000E0001636F000E8B
:10070000626F000E0001656F080E646F4EECABF077
:10071000000120EE01F0AB51D926AC51DA22DF50B6
:100720000001B16F030E0001B117D8B44CD1ABC0BA
:10073000D9FFACC0DAFFDF500001B76F020E000135
:10074000B96F010E0001BF6F020E0001BA6F28D110
:100750000001BA510001686F696B68BF6907000E3C
:1007600000016B6F010E6A6F32ECABF00001685153
:100770000001AB25D96E000169510001AC21DA6E90
:10078000DF500001B86F0001B85152EC9CF06EC010
:10079000B3F06FC0B4F0000E0001BB6FF3D00001E6
:1007A000BB510001686F696B68BF6907000E0001EB
:1007B0006B6F010E6A6F32ECABF0B3C0B1F0B4C036
:1007C000B2F0000168510001B12700016951000138
:1007D000B223B1C0F6FFB2C0F7FF000EF86E0800FA
:1007E000F5CFBDF0020E0001AD250001606F000ED7
:1007F0000001AE210001616FB8C062F00001636BBF
:10080000000E0001656F060E646FA7ECA6F00001F4
:10081000605100016111D8A402D0010E01D0000E78
:100820000001BE6F7FD0ABD00001BE510001D8B433
:10083000A6D09AEC97F047D0A2D00001BE5100019B
:10084000D8B49DD011ECACF03ED099D00001BE518F
:100850000001D8B494D07DECACF035D090D000013C
:10086000BE510001D8B48BD047ECACF02CD087D06F
:100870000001BE510001D8B482D06BECACF023D0A3
:100880007ED00001BE510001D8B479D023ECACF089
:100890001AD075D00001BE510001D8B470D059EC07
:1008A000ACF011D06CD00001BE510001D8B467D0BB
:1008B00035ECACF008D063D00001BE510001D8B4D3
:1008C0005ED0FFECABF0040E0001BF6F58D000010A
:1008D000B78155D00001B78952D00001B7834FD0FE
:1008E0000001B78B4CD0ABC0D9FFACC0DAFFDF50F2
:1008F0000001686FBEC069F00001BD5151ECA5F068
:100900000001BD6F0001B951010DF3500001AF2589
:10091000D96EF4500001B021DA6EBDC0DFFF0001D6
:10092000B92B2DD00001BD51000AD8B428D03A0A05
:10093000D8B47AD7010AD8B480D7070AD8B486D7F2
:10094000010AD8B48CD7030AD8B492D7010AD8B414
:1009500098D77F0AD8B49ED7010AD8B4A4D7030A7F
:10096000D8B4AAD7A20AD8B4B2D7010AD8B4B5D796
:10097000050AD8B4AFD7010AD8B4B2D7B4D70001AA
:10098000BB2B00D00001BB51800A7D0FD8B005D031
:10099000070E0001B96503D700D00001BA2B00D0C3
:1009A0000001BA51800A780FD8B006D00001BF0507
:1009B000D8A402D0CDD600D0AFC0D9FFB0C0DAFFE6
:1009C000B7C0DFFF29D0ABC060F0ACC061F0C6ECAF
:1009D000A5F00009D8B40FD0ABC0A5F0ACC0A6F00C
:1009E000ADC0A7F0AEC0A8F0AFC0A9F0B0C0AAF0EB
:1009F00060EC91F00ED0ABC073F0ACC074F0ADC041
:100A000075F0AEC076F0AFC077F0B0C078F03FECD4
:100A100098F00001BF6F00D0040E0001F4619DD07A
:100A20000001F751D8B499D0000120EE01F0AD518A
:100A3000D926AE51DA22DF500001B16F000120EE5D
:100A400001F0AB51D926AC51DA22DF500001B119C7
:100A50000001B26F030E0001B217D8B46AD00001D2
:100A600020EE01F0AB51D926AC51DA22DF50030B56
:100A70000101CF6F0101CF510101D8B403D0CFC123
:100A800057F057D05750D8B454D00001BF05D8A460
:100A900050D0000120EE02F0AF51D926B051DA2239
:100AA000DF50D8A446D057B205D0000E0001B66F73
:100AB000910E04D0000E0001B66F900EB56F00D0FD
:100AC000B5C0BCF0ABC0D9FFACC0DAFFDF5000014D
:100AD000686F010E0001696F0001BC5151ECA5F077
:100AE0000001BC6F000120EE02F0AF51D926B051D9
:100AF000DA22BCC0DFFFADC060F0AEC061F0ABC0B9
:100B000062F0ACC063F0000E0001656F080E646F08
:100B100060EC9BF0000120EE01F0AD51D926AE5102
:100B2000DA225750DF12000E576E0001BF5112003B
:100B300000D05750D8B411D00001BF05D8A40AD0B6
:100B4000000120EE02F0AF51D926B051DA22DF5079
:100B5000D8B403D0000E576E00D00001BF05D8B442
:100B60000AD0030E0001BF19D8B405D0040E00014D
:100B7000BF19D8A410D0ADC060F0AEC061F0ABC05A
:100B800062F0ACC063F0000E0001656F080E646F88
:100B900060EC9BF000D00001BF5112001200000E6B
:100BA0000001C46F3CEC9DF00009D8B410D0CAD14C
:100BB0000ED00001F051010DDF0EF324D96E010EAD
:100BC000F420DA6E0E0EDF6E0001F02B00D0000173
:100BD000F051800A780FD8A0ECD70001F251080D2F
:100BE000400EF3240001606F020EF4200001616FDB
:100BF000DF0E0001626F010E0001636F000E000145
:100C0000656F080E646F60EC9BF00001F151000805
:100C10000001F225060F0001C76F0001C751800ACD
:100C20007A0FD8A003D0FA0E0001C7270001C751E0
:100C3000050F0001C96F0001C951800A7A0FD8A0C1
:100C400004D0FA0E0001C92700D0020E0001F06F97
:100C5000020E0001C86F0001C851800A780FD8B099
:100C60005FD001D05DD00001C751080D400E0001DA
:100C7000C26F020E0001C36FF3500001C227F4508F
:100C80000001C3230001C851010DF3500001C2252A
:100C9000D96EF4500001C321DA6EDF500001C56F38
:100CA0000001C951080D020EF326000EF422400E79
:100CB000F3240001606F020EF4200001616FC5C0D3
:100CC00062F00001636B000E0001656F060E646F39
:100CD000A7ECA6F00001605100016111D8B40ED05C
:100CE0000001F051010DDF0EF324D96E010EF42046
:100CF000DA6EC5C0DFFF0001F02B00D00001C82B69
:100D0000AAD70ED00001F051010DDF0EF324D96EE9
:100D1000010EF420DA6E0E0EDF6E0001F02B00D013
:100D20000001F051800A780FD8A0ECD70001F251F1
:100D3000050F0001C96F0001C951800A7A0FD8A0C0
:100D400004D0FA0E0001C92700D00001C951080DD6
:100D5000400EF324D96E020EF420DA6EDF5000014B
:100D6000C26F0001F251080D400EF324D96E020E3D
:100D7000F420DA6EDF500001C2150101DF6F0001BF
:100D8000C951080D010EF326000EF422400EF32483
:100D9000D96E020EF420DA6EDF500001C26F00013E
:100DA000F251080D010EF326000EF422400EF3243A
:100DB000D96E020EF420DA6EDF500001C215010177
:100DC000E06F0101CEA503D00101E08100D0DFC1B9
:100DD000C6F00001F851D8B420D0DF0E0001606FDA
:100DE000010E0001616FC6ECA5F00009D8B415D062
:100DF0005A500101DF130101D2B306D00001C6A38E
:100E000003D0020E5A1A00D00101D2BB06D0000155
:100E1000C6AB03D0200E5A1A00D0C6C0D2F1DF0EE6
:100E20000001606F010E0001616FE70E0001626F4B
:100E3000010E0001636F000E0001656F080E646F04
:100E40008EECA4F00001605100016111D8B473D0A0
:100E5000E10E0001606F010E0001616FE90E0001FB
:100E6000626F010E0001636F000E0001656F060ED8
:100E7000646F8EECA4F00001605100016111D8A4F0
:100E800010D00E0E0101E119D8B40BD00101E051D0
:100E9000D8A407D0DFC1C2F0220E0001C217D8B417
:100EA0001BD00E0E0101E119D8B403D0000E5A6E0A
:100EB00000D0DF0E0001AB6F010E0001AC6FE70E3A
:100EC0000001AD6F010E0001AE6FC0C0AFF0C1C038
:100ED000B0F061EC83F02CD00101E851D8B404D01B
:100EE0000101E051D8B427D00001F751D8B40ED099
:100EF0000101E7A303D00101DFA31DD00101E7AB8E
:100F000005D00101DFAB17D001D015D0DF0E0001F5
:100F1000AB6F010E0001AC6FE70E0001AD6F010E6B
:100F20000001AE6FC0C0AFF0C1C0B0F061EC83F0A3
:100F30000001C46F00D0C0C06EF0C1C06FF0E6EC1D
:100F400087F02DD00001F251050F0001C96F00019B
:100F5000C951800A7A0FD8A004D0FA0E0001C9271F
:100F600000D00001F251080D400EF3240001606F23
:100F7000020EF4200001616F0001C951080D400EFE
:100F8000F3240001626F020EF4200001636F000E73
:100F90000001656F080E646F60EC9BF000D00001EB
:100FA000F22B0001F251800A7A0FD8A003D0000E74
:100FB0000001F26F020E0001F06F000E0101E06F00
:100FC000E0C1DFF10001C45112001200020E000165
:100FD000716F00017151800A780FD8B0120001D0F2
:100FE0001200000171510001686F696B68BF6907E9
:100FF000000E00016B6F010E6A6F32ECABF0000166
:10100000685100016E25D96E0001695100016F2100
:10101000DA6EDF500001706F99D1B6D13DD000017A
:1010200071510001686F696B68BF6907000E0001AC
:101030006B6F010E6A6F32ECABF00001685100017A
:101040006E25D96E0001695100016F21DA6E2C0EF8
:10105000CCD06EC0D9FF6FC0DAFF030EDF1294D17F
:10106000000171510001686F696B68BF6907000E6C
:1010700000016B6F010E6A6F32ECABF0000168513A
:1010800000016E25D96E0001695100016F21DA6EF1
:101090002A0EABD0DED778D100017051900AD8B4B7
:1010A000BED7010AD8B4DCD76FD122D000D000015E
:1010B00071510001686F696B68BF6907000E00011C
:1010C0006B6F010E6A6F32ECABF0000168510001EA
:1010D0006E25D96E0001695100016F21DA6E350E5F
:1010E000D1D06EC0D9FF6FC0DAFF000EDB844CD1C7
:1010F00000017051900AD8B4DAD7010AD8B4D7D712
:1011000043D135D0000171510001686F696B68BF30
:101110006907000E00016B6F010E6A6F32ECABF0D5
:101120000001685100016E25D96E0001695100016E
:101130006F21DA6E8A0E80D0000171510001686F54
:10114000696B68BF6907000E00016B6F010E6A6F63
:1011500032ECABF00001685100016E25D96E000140
:10116000695100016F21DA6E8B0E66D00DD100013E
:101170007051900AD8B4C6D7010AD8B4DDD704D1CB
:1011800037D0000171510001686F696B68BF690752
:10119000000E00016B6F010E6A6F32ECABF00001C4
:1011A000685100016E25D96E0001695100016F215F
:1011B000DA6E8A0E1AD04DD7000171510001686FA6
:1011C000696B68BF6907000E00016B6F010E6A6FE3
:1011D00032ECABF00001685100016E25D96E0001C0
:1011E000695100016F21DA6E8B0EDF6E32D7CCD0E1
:1011F00000017051900AD8B4C4D7010AD8B4DCD722
:10120000C3D01CD000D0000171510001686F696B20
:1012100068BF6907000E00016B6F010E6A6F32EC48
:10122000ABF00001685100016E25D96E00016951D3
:1012300000016F21DA6E350EDF6EA6D0000170510D
:10124000900AD8B4E0D7010AD8B4DDD79DD01DD01C
:1012500000D0000171510001686F696B68BF6907B8
:10126000000E00016B6F010E6A6F32ECABF00001F3
:10127000685100016E25D96E0001695100016F218E
:10128000DA6E2C0EDF6E2DD77FD000017051900AE0
:10129000D8B4DFD7010AD8B4DCD776D022D000D0BA
:1012A000000171510001686F696B68BF6907000E2A
:1012B00000016B6F010E6A6F32ECABF000016851F8
:1012C00000016E25D96E0001695100016F21DA6EAF
:1012D0002C0EDF6E6EC0D9FF6FC0DAFF000EDB820E
:1012E00053D000017051900AD8B4DAD7010AD8B4AB
:1012F000D7D74AD022D000D0000171510001686FC9
:10130000696B68BF6907000E00016B6F010E6A6FA1
:1013100032ECABF00001685100016E25D96E00017E
:10132000695100016F21DA6E2C0EDF6E6EC0D9FF9D
:101330006FC0DAFF000EDB8027D000017051900AE9
:10134000D8B4DAD7010AD8B4D7D71ED00001F751E4
:10135000010AD8B419D0030AD8B49ED6010AD8B469
:10136000C7D6070AD8B403D7010AD8B441D7030AAD
:10137000D8B464D7010AD8B488D70F0AD8B4B1D783
:10138000010AD8B4DAD700D00001712B22D612009E
:101390000001816FA10E000181619BD081C060F0CE
:1013A0000001616B000E0001636F070E626F5DEC60
:1013B0009FF0D8900001603700016137BC0E00013A
:1013C000602500017F6FFD0E000161210001806F2B
:1013D000000E0001826F24D000018251010D7FC0F8
:1013E0007AF080C07BF0F35000017A27F4500001BE
:1013F0007B237AC0F6FF7BC0F7FF000EF86E00017A
:101400008251010DF35000017825D96EF45000018E
:101410007921DA6E0800F5CFDFFF0001822B00D0C2
:10142000020E000182611AD000018251010D7FC0BD
:101430007AF080C07BF0F35000017A27F45000016D
:101440007B237AC0F6FF7BC0F7FF000EF86E080022
:10145000F5500009D8B402D0BFD700D081C060F0E9
:101460000001616B000E0001636F070E626FACEC50
:10147000A1F0750E00016025F66EF70E00016121E6
:10148000F76EF86A000EF82200018251010DF35048
:1014900000017825D96EF45000017921DA6E080038
:1014A000F5CFDFFF0DD000018251010DF350000197
:1014B0007825D96EF45000017921DA6E000EDF6EC6
:1014C0000001822B00D0020E00018265ECD71200D1
:1014D0001200A00E000181652AD0B70E00018161C3
:1014E00026D078C06EF079C06FF05F0E00018125C4
:1014F0000001686F0001696BFF0E6923000E000197
:101500006B6F030E6A6F32ECABF0980E000168252A
:101510000001706FFC0E000169210001716F000E67
:101520000001736F030E726F10ECA7F01200C70E6C
:10153000000181653AD0E20E0001816136D078C0A9
:101540006EF079C06FF0700E00017A6FFE0E000130
:101550007B6F0001815100017C6F7D6BD890000191
:101560007C377D3700017A5100017C2700017B51D7
:1015700000017D23560E00017C250001706FFD0ED9
:1015800000017D210001716F000E0001736F020EDA
:10159000726F10ECA7F0000120EE02F07851D9260E
:1015A0007951DA22000EDF6E1200E50E000181652E
:1015B0009AD0F20E0001816196D0000181511A0F7C
:1015C0000001826F28D000018251030D850EF324A3
:1015D00000017F6FFE0E1BD000018251030D3D0EF6
:1015E000F32400017F6FFE0E12D000018251030D23
:1015F000610EF32400017F6FFE0E09D000D00001C0
:101600008251030DCD0EF32400017F6FFE0EF420F6
:101610000001806F0FD00001F351000AD8B4EFD75A
:10162000010AD8B4E2D7030AD8B4CDD7010AD8B496
:10163000D3D7E5D7000E0001826F020E000182654C
:1016400002D01200120000018251010D7FC07AF019
:1016500080C07BF0F35000017A27F45000017B2317
:101660007AC0F6FF7BC0F7FF000EF86E0800F5CFDA
:101670007EF0D7ECABF00009D8A40ED01FD00CD070
:10168000300E07D0320E05D02E0E03D0250E01D01D
:10169000260E00017E6F12D000017E51260AD8B4BA
:1016A000F5D7010AD8B4F4D7080AD8B4E9D71F0A85
:1016B000D8B4E8D7050AD8B4E7D700D000018251E2
:1016C000010DF35000017825D96EF4500001792105
:1016D000DA6E7EC0DFFF0001822B020E0001826500
:1016E000B2D71200120078C060F079C061F0000E2D
:1016F0000001636F000E626F000E0001656F030E44
:10170000646F4EECABF01200FE0EF66E1F0EF76E1D
:10171000000EF86E0900060EF55E0900000EF55A7F
:10172000D8A070D0000E0001626F070E0001626544
:1017300001D02DD000016251020D500EF324D96E5C
:10174000010EF420DA6E00016251020D300EF32416
:10175000E16E010EF420E26EDECFE6FFDDCFE5FFA5
:1017600000016251010DA80EF324D96E010EF42080
:10177000DA6E00016251010D900EF324E16E010E4C
:10178000F420E26EDFCFE7FF0001622BCED7000E20
:101790000001636F0B0E0001636502D0120012009E
:1017A00000016351020D700EF324D96E020EF42075
:1017B000DA6E00016351020D000EF324E16E010E9A
:1017C000F420E26EDECFE6FFDDCFE5FF00016351DE
:1017D000010D840EF324D96E010EF420DA6E00019F
:1017E0006351010D600EF324E16E010EF420E26EF0
:1017F000DFCFE7FF0001632B0B0E00016365D0D73D
:1018000012001200FE0EF66E1F0EF76E000EF86E3E
:101810000900040EF55E0900000EF55AD8A07FD02D
:10182000000E0001646F070E0001646501D02DD029
:1018300000016451020D400EF324D96E010EF42014
:10184000DA6E00016451020D300EF324E16E010ED8
:10185000F420E26EDECFE6FFDDCFE5FF000164514C
:10186000010DA00EF324D96E010EF420DA6E0001F2
:101870006451010D900EF324E16E010EF420E26E2E
:10188000DFCFE7FF0001642BCED7000E0001656FAC
:101890000B0E0001656501D02DD000016551020DD0
:1018A000180EF324D96E010EF420DA6E0001655192
:1018B000020D000EF324E16E010EF420E26EDECF85
:1018C000E6FFDDCFE5FF00016551010D780EF32441
:1018D000D96E010EF420DA6E00016551010D600E23
:1018E000F324E16E010EF420E26EDFCFE7FF00018A
:1018F000652BCED7FE0EF66E1F0EF76E000EF86E3D
:101900000900050EF55E0900000EF55AD8A0120078
:10191000010E01016A6F020E01016B6F1200FE0ED3
:10192000F66E1F0EF76E000EF86E0900030EF51826
:101930000900F510D8A41200960E01013A6F0F0E9F
:1019400001013B6F000E0001606F070E0001606532
:1019500001D017D000016051010D980EF324D96E0B
:10196000010EF420DA6E00016051010D900EF32497
:10197000E16E010EF420E26EDFCFE7FF0001602B85
:10198000E4D7000E0001616F0B0E0001616502D00B
:101990001200120000016151010D6C0EF324D96E8A
:1019A000010EF420DA6E00016151010D600EF32486
:1019B000E16E010EF420E26EDFCFE7FF0001612B44
:1019C0000B0E00016165E6D7120012001200030E33
:1019D0005F18D8A42DD0C3ECABF00001D06F000E7F
:1019E0000001CF6FC40E0001D019D8A406D0220E7A
:1019F0000001D06F020E0001CF6F05010251D8B473
:101A00000AD00001D05105010219D8A404D0000E5B
:101A10000501026F1FD114ECAAF0D0C002F5CFC0AF
:101A200000F505010251D8A415D1000E5F6E12D148
:101A300006ECA8F00009D8B496D0F19E968EEF0E71
:101A40009312CE0E95122F0E9212070E961200D000
:101A5000070E0001D36F79D00001D351010D900E14
:101A6000F324D96E010EF420DA6EDF50FF0A000174
:101A7000CC6F0001D351020D300EF324D96E010E4C
:101A8000F420DA6EDECFCDF0DDCFCEF0CDC0D9FFC1
:101A9000CEC0DAFF0001CC51DF16000E0001D26F7C
:101AA0000B0E0001D26501D02DD00001D251010DE5
:101AB000600EF324D96E010EF420DA6EDF500001BF
:101AC000CC6F0001D251020D000EF324D96E010E2D
:101AD000F420DA6EDECFCDF0DDCFCEF0CDC0D9FF71
:101AE000CEC0DAFFDF500001CC150009D8A407D022
:101AF000D2C073F00001D35188EC8FF000D0000108
:101B0000D22BCED70001D351010D900EF324D96E04
:101B1000010EF420DA6EDF500001CC6F0001D351CA
:101B2000020D300EF324D96E010EF420DA6EDECFF2
:101B3000CDF0DDCFCEF0CDC0D9FFCEC0DAFF0001B1
:101B4000CC51DF120001D30700D00001D3AF84D7FE
:101B5000969EF18ED00E9216F80E9616100E9316D3
:101B6000310E951600D0000E0001C06F050E000169
:101B7000C16FCFEC85F05F6E5FD0100E0001606F1B
:101B8000050E0001616F000E0001636F000E626FB1
:101B9000000E0001656F060E646F4EECABF05AD07C
:101BA000000E0001D16F050E0001D16501D00FD0EC
:101BB0000001D151010D020EF324D96E050EF4205F
:101BC000DA6EDF50A7ECA9F00001D12BECD7060E9E
:101BD0004FECADF00501026F030E0001606F050EC2
:101BE0000001616F000E0001636F000E626F000E56
:101BF0000001656F050E646F4EECABF02BD0030E49
:101C00005F6E000E0501006FFE0E4FECADF005019A
:101C1000026F030E0001606F050E0001616F000E80
:101C20000001636F000E626F000E0001656F050E0C
:101C3000646F4EECABF00ED05F50010AD8B40AD0FE
:101C4000030AD8B49AD7010AD8B4AAD7070AD8B4D5
:101C5000D6D700D05F50D8A407D0000E0001CA6FBD
:101C6000000E0001CB6F1200000E0001CA6F050EBE
:101C70000001CB6F120012000D012205D8A412D072
:101C80000D0120511F0B0009D8A40CD00001FC8FBE
:101C9000030E0D012119D8A402D0010E01D0000EAF
:101CA000526E00D00D012251D8A412000D01205116
:101CB0001F0B020AD8A412000D0124510F0B0009BA
:101CC000D8B412000D0124510F0B366E020E36608F
:101CD0001200200E0001EF19D8A412000001FC8FA1
:101CE0000D0124BF1BD00D0124510F0B366E365051
:101CF000020DBD0EF324D96E010EF420DA6EDECF94
:101D00003AF0DDCF3BF00D0124510F0B366E36500B
:101D1000010DEB0EF324D96E000E1AD00D012451E3
:101D20000F0B366E3650020DE50EF324D96E000E01
:101D3000F420DA6EDECF3AF0DDCF3BF00D01245116
:101D40000F0B366E3650010DE90EF324D96E000EDE
:101D5000F420DA6EDF50396E00D039B002D03A94F8
:101D600002D03A8400D00D0124BF0BD00D012451C4
:101D70000F0B366E3650020DBD0EF324D96E010ED8
:101D80000AD00D0124510F0B366E3650020DE50EB0
:101D9000F324D96E000EF420DA6E3AC0DEFF3BC0A9
:101DA000DDFF00D0030E0D012119D8A430D03AC0B8
:101DB000D9FF3BC0DAFFDFAE1DD00D0124BF0BD031
:101DC0000D0124510F0B366E3650010DEB0EF3242E
:101DD000D96E000E0AD00D0124510F0B366E36500D
:101DE000010DE90EF324D96E000EF420DA6E000125
:101DF000DF8200D03AC0D9FF3BC0DAFF000EDB849F
:101E00003AC0D9FF3BC0DAFF000EDB8E1200040E91
:101E10003A1A3AC0D9FF3BC0DAFFDFAE1BD03AC056
:101E2000D9FF3BC0DAFF7F0EDF163AC0D9FF3BC0B7
:101E3000DAFF000EDB8C000E2F6E050E2E6E3AC000
:101E400030F03BC031F0000E336E020E326E38ECD3
:101E5000A6F007D03AC0D9FF3BC0DAFF000EDB8CFA
:101E600000D0040E3A1A39B206D03AC0D9FF3BC0AE
:101E7000DAFFDFAE32D00D0124BF0BD00D012451AB
:101E80000F0B366E3650010DEB0EF324D96E000E9B
:101E90000AD00D0124510F0B366E3650010DE90E9C
:101EA000F324D96E000EF420DA6E0001DF9200D028
:101EB0003AC0D9FF3BC0DAFF3B0EDF16000E2F6E93
:101EC000050E2E6E3AC030F03BC031F0000E336E7E
:101ED000020E326E38ECA6F007D03AC0D9FF3BC0F4
:101EE000DAFF3B0EDF1600D00D0124510F0B366ECA
:101EF0003650010D260EF324376E0F0EF420386E87
:101F000037C0D9FF38C0DAFFFE0EDF16120012000C
:101F10000001786F00017351010DD30EF324D96EC7
:101F2000010EF420DA6EDF2A00017851010DEF0E68
:101F3000F324D96E010EF420DA6EDF2AFE0EF66E5F
:101F40001F0EF76E000EF86E0900020EF55E090016
:101F5000000EF55AD8B009D0000178510C0DF3509D
:101F6000000173250001776F40D0000178510C0DFE
:101F7000E70E0001746FF40E0001756FF35000015D
:101F80007427F4500001752300017351010DF350C3
:101F900000017427F4500001752374C0F6FF75C06A
:101FA000F7FF000EF86E0800F5CF77F077C060F00D
:101FB0000001616B000E0001636F0C0E626F5DEC3F
:101FC0009FF0000160510001786F77C060F0000160
:101FD000616B000E0001636F0C0E626FACECA1F040
:101FE000000160510001736F00D0070E00017819E5
:101FF000D8A42FD0F4C074F0030E000174170001B0
:1020000074510C0D270E0001756FF70E0001766FED
:10201000F35000017527F45000017623000173513D
:10202000010DF35000017527F4500001762375C0AF
:10203000F6FF76C0F7FF000EF86E0800F5CF73F0DC
:10204000000178510C0DF350000173250001776FEA
:1020500000D000017751CFEC98F00001796FDF0ECE
:10206000000179651AD0E80E0001796116D079C0B7
:1020700074F0200E00017427010E0001756F00013D
:10208000742B03D00001D89075370001742FFAD754
:10209000000175510101DF131200EF0E0001796597
:1020A0001AD0F20E0001796116D079C074F0100ECA
:1020B00000017427010E0001756F0001742B03D01D
:1020C0000001D89075370001742FFAD700017551BF
:1020D0000101E01312000001F051800A780FD8B01E
:1020E00012000001F051010DDF0EF324D96E010E34
:1020F000F420DA6E77C0DFFF0001F02B120012002F
:102100000001FF69000E0001826F00018251800A08
:10211000700FD8B04CD001D04AD0000182510001DC
:10212000686F696B68BF6907000E00016B6F400E36
:102130006A6F32ECABF0000168C07EF0000169C04C
:102140007FF0000E00017FBFFF0E806F816F000ED9
:1021500000017E2500016E6FF80E00017F21000155
:102160006F6F010E000180210001706F000E0001F1
:1021700081210001716F000E0001736F400E726FBC
:10218000000E0001746F020E0001756FDEECA6F008
:1021900002013F05D8A40BD0040E02013E6107D016
:1021A00082C0FFF001D003D00001822BAED7000126
:1021B000FF29D8A448D00F0E0001FF6F000E0201C6
:1021C0003E6F000E0001836F00018351800A7C0F77
:1021D000D8B0120001D01200000183510A0D000E88
:1021E000F32400016E6F020EF42000016F6FC30E26
:1021F0000001706FFF0E0001716F000E0001736F20
:10220000080E726F10ECA7F0000183510A0D080E42
:10221000F326000EF422000EF3240001606F020E7C
:10222000F4200001616F000E0001636F000E626F09
:10223000000E0001656F020E646F4EECABF0000102
:10224000832BC2D712000001FF510001686F696B38
:1022500068BF6907000E00016B6F400E6A6F32ECB9
:10226000ABF0000168C07EF0000169C07FF0000E95
:1022700000017FBFFF0E806F816F000E00017E2581
:1022800000016E6FF80E00017F2100016F6F010EDB
:10229000000180210001706F000E0001812100010A
:1022A000716F000E0001736F400E726F000E00011F
:1022B000746F020E0001756FDEECA6F012001200C2
:1022C000B4D0A5C083F0A6C084F0A7C085F0A8C094
:1022D00086F0A9C087F0AAC088F0F40E0001896FCB
:1022E000FA0E00018A6F480E00018B6FFB0E000191
:1022F0008C6F9C0E00018D6FFB0E00018E6F00EC49
:1023000080F01200A5C083F0A6C084F0A7C085F0BD
:10231000A8C086F0A9C087F0AAC088F0500E0001BE
:10232000896FF90E00018A6FA40E00018B6FF90E00
:1023300000018C6FF80E00018D6FF90E00018E6F99
:1023400000EC80F01200A5C083F0A6C084F0A7C006
:1023500085F0A8C086F0A9C087F0AAC088F0A80EB2
:102360000001896FF80E00018A6FFC0E00018B6F6F
:10237000F80E00018C6FFC0E00018D6FF80E00014D
:102380008E6F00EC80F01200A5C083F0A6C084F030
:10239000A7C085F0A8C086F0A9C087F0AAC088F0C1
:1023A0004C0E0001896FFA0E00018A6FA00E000129
:1023B0008B6FFA0E00018C6FA00E00018D6FFA0E6C
:1023C00000018E6F00EC80F01200A5C083F0A6C063
:1023D00084F0A7C085F0A8C086F0A9C087F0AAC085
:1023E00088F0F00E0001896FFB0E00018A6F440E29
:1023F00000018B6FFC0E00018C6F440E00018D6F8D
:10240000FC0E00018E6F00EC80F01200A5C073F08E
:10241000A6C074F0A7C075F0A8C076F0A9C077F088
:10242000AAC078F03FEC98F012000001F551010AC3
:10243000D8B468D7030AD8B444D7010AD8B4A4D70B
:10244000070AD8B4C2D7010AD8B47DD7DFD71200A3
:10245000A098000E636E000E626E000E0F01266FD4
:10246000270E0001606F0F0E0001616F000E00016A
:10247000636F000E626F000E0001656F010E646FE6
:102480004EECABF0160E0F01396F9F0E0F01376F38
:102490007B0E0F01366F000E0001686F10D013D055
:1024A00000016851040D000EF324D96E0D0EF420C6
:1024B000DA6EDE6ADE6ADE6ADD6A0001682B070E0C
:1024C00000016865EDD7658C000E0F01386F6598C7
:1024D000659C0DD06296000E0001FC6F000E00019D
:1024E000DF6F000E0001E16F000EE06F00D062B6FA
:1024F000F1D7010E0101CA6F010E0101CB6F000E71
:102500000101C86F000E0101C96F000E536E000E6D
:102510000001686F010E0001686501D033D0000131
:102520006851020DE50EF324D96E000EF420DA6E28
:10253000000EDE6E000EDD6E00016851020DBD0E54
:10254000F324D96E010EF420DA6E000EDE6E000E5A
:10255000DD6E00016851010DE90EF324D96E000E05
:10256000F420DA6E000EDF6E00016851010DEB0EF3
:10257000F324D96E000EF420DA6E000EDF6E000137
:10258000682BC8D7080E0001E56F0D0E0001E66F3D
:10259000160E0F01266F0D0E0D01036F200E026F38
:1025A000080E0D01016F040E0D01006F0D01008F6B
:1025B000000E5C6E000E0001EF6F12000001EF05CF
:1025C000D8B465BA0AD0000E626E0F0136810F01D1
:1025D0003689020E0001EF6F00D062A407D00F0110
:1025E00036A504D06294F6ECAAF000D065A202D021
:1025F000A198120062A00BD00F0136A108D04DECBB
:1026000096F0A088040E0001EF6F629000D062A8DF
:1026100007D00F0136A904D0AEECABF0629800D021
:1026200062AC1ED00F0136AD0FD0000E2F6E730EB0
:102630002E6E000E306E000E316E000E336E010EE7
:10264000326E38ECA6F000D0629C5550D8B402D05F
:10265000550600D05550D8A403D08CEC9EF000D085
:1026600062AA06D00F0136AB03D0F0ECA9F000D07F
:1026700062A213D00F0136A310D07F0E2F6E2E68EA
:10268000000E306E000E316E000E336E010E326E93
:1026900038ECA6F0000E636E00D0040E0001EF616E
:1026A00002D0A19812000F0136A73CD0000E3F6E59
:1026B000030E3F6401D036D062A634D064CF5EF002
:1026C0005E30E832E8320F0B586E62965EB407D087
:1026D0005850010DEB0EF324D96E000E06D0585061
:1026E000010DE90EF324D96E000EF420DA6E00011C
:1026F000DF7000D05850D8A403D0C5EC9FF010D0A4
:10270000000E2F6E720E2E6E5E0E306E000E316E4B
:10271000000E336E000E326E38ECA6F001D002D0FF
:102720003F2AC6D7A19812000D0120511F0BE806C1
:10273000D8A4120001D012000D012451D8A4120017
:1027400001D01200060E0D012119D8B42CD035D0BD
:102750002AD05C04D8A431D00D012451D8A42DD0A6
:10276000260E0001F96FFE0E0001FA6F000E000147
:10277000FE6F090E15D0C00E0001FC6F1ED05C0468
:10278000D8A41BD00D012451D8A417D0DA0E000113
:10279000F96FFC0E0001FA6F000E0001FE6F400E93
:1027A000FD6FE9D70AD00D012351210AD8B4D1D742
:1027B000030AD8B4E4D7010A00D00D012039E83269
:1027C000030BE806D8A412004CD012004AD0120025
:1027D00069ECABF012000D012451010DFE0EF32443
:1027E0000001F96F010EF4200001FA6F000E0001E4
:1027F000FE6F010EFD6FC10E0001FC6F1200800E16
:102800000001FC6F0D012451010DFE0EF324D96E61
:10281000010EF420DA6E23CDDFFF12000D012451EA
:10282000010DFD0EF3240001F96F010EF4200001EB
:10283000FA6F000E0001FE6F010EFD6F810E0001A8
:10284000FC6F1200800E0001FC6F0D012451010D80
:10285000FD0EF324D96E010EF420DA6E22CDDFFFD7
:1028600012000D012151010AD8B41200030AD8B494
:10287000B2D7010AD8B4D2D70A0AD8B4A9D7030A62
:10288000D8B4BDD7010AD8A41200DCD7120000D0FA
:10289000C3C1D4F0C4C1D5F00001D41FD51FD44B9F
:1028A000D52B64ECADF00001D4510001602700018C
:1028B000D55100016123000161BFEAD7190E000163
:1028C000605D010E00016159D8A0E2D764ECADF063
:1028D00060C0C3F161C0C4F10101C52BC5C1D4F012
:1028E0000001D56BD4BFD5070001D4B1120001D0CF
:1028F00012000101B9510101BA11D8B413D0B9C104
:10290000D9FFBAC1DAFF0101DFAE04D00001D46BF8
:10291000D42B02D00001D46B0001D4510001D66F3A
:10292000D76B06D0000E0001D76F000ED66F00D017
:102930000001D6510001D711D8A41ED0E7EC8CF0CD
:10294000CAC0DAF0CBC0DBF00001DA510001DB11C4
:10295000D8B412D0010E0001606FDAC061F0DBC0A4
:1029600062F0080E0001636F010E1DEC9EF060C066
:10297000B9F161C0BAF100D00101BB510101BC1134
:10298000D8B413D0BBC1D9FFBCC1DAFF0101DFAE9F
:1029900004D00001D46BD42B02D00001D46B000111
:1029A000D4510001D86FD96B06D0000E0001D96F49
:1029B000000ED86F00D00001D8510001D911D8A461
:1029C0001200000E0001606F080E0001616F050E1D
:1029D0000001626F010E0001636F010E1DEC9EF09D
:1029E00060C0BBF161C0BCF1120012000001FF69C0
:1029F000000E2A6E2A50800A700FD8B03AD001D04B
:102A000038D02A50106E116A10BE1106000E136ED7
:102A1000400E126EEBECABF010C026F011C027F0A8
:102A2000000E27BEFF0E286E296E000E2624166E9D
:102A3000F80E2720176E010E2820186E000E292090
:102A4000196E000E1B6E400E1A6E000E1C6E020EEA
:102A50001D6E34ECA8F002013F05D8A40AD0040E84
:102A600002013E6106D02AC0FFF001D002D02A2A1E
:102A7000C1D70001FF29D8A43AD00F0E0001FF6F83
:102A8000000E02013E6F000E2B6E2B50800A7C0F51
:102A9000D8B0120001D012002B500A0D000EF32402
:102AA000106E020EF420116EC30E126EFF0E136E26
:102AB000000E156E080E146E62ECA8F02B500A0D75
:102AC000080EF326000EF422000EF324106E020E00
:102AD000F420116E000E136E000E126E000E156EB5
:102AE000020E146E97ECABF02B2ACFD71200000128
:102AF000FF51106E116A10BE1106000E136E400ECB
:102B0000126EEBECABF010C026F011C027F0000EF7
:102B100027BEFF0E286E296E000E2624166EF80EB4
:102B20002720176E010E2820186E000E2920196E1E
:102B3000000E1B6E400E1A6E000E1C6E020E1D6EF5
:102B400034ECA8F012001200800E0D012019D8A458
:102B50001200C00E0001FC6F92D08A0E0001F96FC6
:102B6000FF0E0001FA6F000E0001FE6F120EFD6FE6
:102B700012000D012251D8A449D00D012251020D9D
:102B8000860EF324F66EF70EF420F76EF86A000E48
:102B9000F8220900F5CFF9F00A00F5CFFAF0020E9D
:102BA0000001F925106E000E0001FA21116E10C00F
:102BB000F6FF11C0F7FF000EF86E0E0EF76403D09B
:102BC0000800F55005D0F6CFE9FFF7CFEAFFEF5048
:102BD0000001FD6F030E0001F925106E000E0001CB
:102BE000FA21116E10C0F6FF11C0F7FF000EF86E4B
:102BF0000E0EF76403D00800F55005D0F6CFE9FFBC
:102C0000F7CFEAFFEF500001FE6F1200000E000147
:102C1000FC6F1200030E0D01226129D00D0122511B
:102C2000020D7C0EF324F66EF70EF420F76EF86AB0
:102C3000000EF8220900F5CFF9F00A00F5CFFAF0FE
:102C4000F9C0F6FFFAC0F7FF000EF86E0E0EF7643B
:102C500003D00800F55005D0F6CFE9FFF7CFEAFF23
:102C6000EF50106E10500001FD6FFE6B1200000E51
:102C70000001FC6F1200000E0001FC6F12000D013C
:102C80002351010AD8B469D7030AD8B472D7010A0C
:102C9000D8B4C0D7F0D712001200A098000E636E0F
:102CA000000E626E000E0F01266F270E106E0F0EC3
:102CB000116E000E136E000E126E000E156E010ED8
:102CC000146E97ECABF0160E0F01396F9F0E0F01CB
:102CD000376F7B0E0F01366F000E186E0ED010D0BE
:102CE0001850040D000EF324D96E0D0EF420DA6E88
:102CF000DE6ADE6ADE6ADD6A182A070E1864F0D71B
:102D0000658C000E0F01386F6598659C0DD062963A
:102D1000000E0001FC6F000E0001DF6F000E0001CD
:102D2000E16F000EE06F00D062B6F1D7010E010135
:102D3000CA6F010E0101CB6F000E0101C86F000EBA
:102D40000101C96F000E536E000E186E010E18645B
:102D500001D02ED01850020DE50EF324D96E000ECE
:102D6000F420DA6E000EDE6E000EDD6E1850020DDD
:102D7000BD0EF324D96E010EF420DA6E000EDE6E65
:102D8000000EDD6E1850010DE90EF324D96E000E11
:102D9000F420DA6E000EDF6E1850010DEB0EF324F6
:102DA000D96E000EF420DA6E000EDF6E182ACED730
:102DB000080E0001E56F0D0E0001E66F160E0F0103
:102DC000266F0D0E0D01036F200E026F080E0D0110
:102DD000016F040E0D01006F0D01008F000E5C6E7F
:102DE000000E0001EF6F120020EE01F04E50D926C8
:102DF0004F50DA22DF50116E11500001E05D000EDD
:102E0000E159D8B003D0E0C011F000D0115000015A
:102E1000E05F000EE15B000E106E13D01050010D4C
:102E2000280EF324D96E0D0EF420DA6EDCC0E1FF1B
:102E3000DDC0E2FFDFCFE7FF0001DC4BDD2B102A16
:102E400000D01150105CD8A0E9D70001E05100017A
:102E5000E111D8B432D020EE01F05050D9265150B3
:102E6000DA22080EDF6E20EE02F05050D9265150C3
:102E7000DA22280EDE6E0D0EDD6E4EC0D9FF4FC079
:102E8000DAFFDFBC0DD050C0D9FF51C0DAFF480EC9
:102E9000DF6E50C0D9FF51C0DAFF000EDB8E12008A
:102EA00050C0D9FF51C0DAFF080EDF6E50C0D9FF05
:102EB00051C0DAFF000EDB8E120020EE01F0505000
:102EC000D9265150DA22080EDF6E20EE02F0505063
:102ED000D9265150DA22200EDE6E0D0EDD6E50C066
:102EE000D9FF51C0DAFF040EDF6E50C0D9FF51C0C8
:102EF000DAFF000EDB8E0001E2510001E311000158
:102F0000E411D8B40ED020EEE2F001D80AD00500CA
:102F1000FA6EDE50FD6EDE50FE6EDE50FF6EFA5031
:102F200012000001DF9F5450D8A412008CEC9EF0D8
:102F3000120012009C0E0001616FFF0E0001626F13
:102F400059ECA9F0CB0E0001616FFF0E0001626F1A
:102F500059ECA9F0FE0EF66E1F0EF76E000EF86E1D
:102F60000900F5CF60F00A00F5CF61F015ECABF089
:102F7000A7ECA9F0280EA7ECA9F0D10E0001616F13
:102F8000FF0E0001626F59ECA9F0000E0001616FA5
:102F9000010E606F15ECABF0A7ECA9F0370EA7ECB3
:102FA000A9F0000E0001616F000E606F15ECABF030
:102FB000A7ECA9F0000E0001616F080E606F15EC20
:102FC000ABF0A7ECA9F0280EA7ECA9F0F10E0001D8
:102FD000616FFE0E0001626F59ECA9F0D70E00017F
:102FE000616FFF0E0001626F59ECA9F0A0ECACF02C
:102FF000DB0E0001616FFF0E0001626F59ECA9F05A
:1030000006ECADF0DF0E0001616FFF0E0001626F94
:1030100059ECA9F0D3ECACF0E30E0001616FFF0EA8
:103020000001626F59ECA9F0F5ECACF0E70E00017D
:10303000616FFF0E0001626F59ECA9F0B1ECACF0CA
:10304000EB0E0001616FFF0E0001626F59ECA9F0F9
:10305000E4ECACF0EF0E0001616FFF0E0001626F57
:1030600059ECA9F0C2ECACF0F30E0001616FFF0E59
:103070000001626F59ECA9F08FECACF0120073C044
:10308000D9FF74C0DAFFDF5000017A6F000120EE33
:1030900001F07351D9267451DA220001DFB476D0E1
:1030A000020E0001796F020E00017C6F00017C515D
:1030B000800A780FD8B06AD001D068D000017C5166
:1030C0000001686F696B68BF6907000E00016B6FD4
:1030D000010E6A6F32ECABF00001685100017325FC
:1030E000D96E0001695100017421DA6EDF500001D0
:1030F0007B6F00017B5160ECA2F000017D6F00014D
:103100007D510001D8A407D000017B51CFEC98F08D
:1031100000017D6F00D07AC068F0020E00017525B5
:103120000001606F000E000176210001616F7DC01B
:1031300062F00001636B000E0001656F060E646FA4
:10314000A7ECA6F00001605100016111D8A402D0E3
:10315000010E01D0000E0001696F00017D5151EC9C
:10316000A5F000017D6F00017951010DF3500001C0
:103170007725D96EF45000017821DA6E7DC0DFFF2B
:103180000001792B00017C2B91D700D077C0D9FFAB
:1031900078C0DAFF7AC0DFFF010E120012000001D2
:1031A0006F6F00016F5160ECA2F00001706F6FC093
:1031B00060F00001616B000E0001636F0C0E626F26
:1031C0005DEC9FF0000160510001716F6FC060F015
:1031D0000001616B000E0001636F0C0E626FACECBE
:1031E000A1F0000160510001726F000170510001F7
:1031F000D8B447D000017051120043D020D0000154
:1032000071510C0DA70E00016D6FF50E1FD000015E
:1032100071510C0D470E00016D6FF50E17D00001B6
:1032200071510C0D070E00016D6FF60E0FD00001ED
:1032300071510C0D670E00016D6FF60E07D0000185
:1032400071510C0DC70E00016D6FF60E00016E6F0F
:10325000F35000016D27F45000016E2300017251FC
:10326000010DF35000016D27F45000016E236DC075
:10327000F6FF6EC0F7FF000EF86E0800F5CF70F095
:1032800012D00001EE51000AD8B4D9D7010AD8B43F
:10329000B6D7030AD8B4BBD7010AD8B4C0D7070A37
:1032A000D8B4C5D7CCD70001705142ECA7F01200BA
:1032B000120065980001FCBF3ED00001DFAF10D0C6
:1032C000020E566E0101C951D8A403D008ECA3F038
:1032D00000D0000E0101CB6F000E0101CA6F120079
:1032E00020EE01F05050D9265150DA22080EDF6E40
:1032F00020EE02F05050D9265150DA22200EDE6E18
:103300000D0EDD6E50C0D9FF51C0DAFF0C0EDF6E1E
:1033100050C0D9FF51C0DAFF000EDB8EE5C0D9FFE7
:10332000E6C0DAFF040EDF6EE5C0D9FFE6C0DAFFC3
:10333000000EDB8E12000D0120AF15D0010E566E6F
:103340000101C851D8A403D008ECA3F000D0000EAE
:103350000101CB6F000E0101CA6F5450D8A41200B6
:103360008CEC9EF01200020E566E20EE01F05050D2
:10337000D9265150DA22080EDF6E20EE02F05050AE
:10338000D9265150DA22200EDE6E0D0EDD6E50C0B1
:10339000D9FF51C0DAFF040EDF6E50C0D9FF51C013
:1033A000DAFF000EDB8E000E0101CB6F000E010173
:1033B000CA6F5450D8A412008CEC9EF01200120078
:1033C000000E0001796F000E00017A6F060E0001F9
:1033D000756FD8900001713370336F336E33000115
:1033E000752FF7D70001060ED8906E376F377037FC
:1033F0007137E82EF9D76EC07BF06FC07CF070C0DB
:103400007DF071C07EF05AD07BC076F07CC077F042
:103410007DC078F0400E0001796F18D073C0D9FFDD
:1034200074C0DAFFDF5076C0F6FF77C0F7FF78C0D0
:10343000F8FFF56E0C000001734B742B0001010EB8
:103440007627000E7723000E782300D0000179073D
:1034500000017929D8A4E2D77BC076F07CC077F050
:103460007DC078F0A684F2AE04D0F29E010E000179
:103470007A6F550EA76EAA0EA76EA682A6940001BB
:103480007A510001D8B405D0F28E000E00017A6F97
:1034900000D0400E00017B2500017B6F000E000173
:1034A0007C2100017C6F000E00017D2100017D6FF9
:1034B000000E00017E2100017E6F00D00001720726
:1034C00000017229D8A4A0D712000D012039E832DA
:1034D000030B0009D8A4120053D0120051D00001F0
:1034E000FC8F080E0001EF6F1200A4EC95F01200A3
:1034F000C8EC9CF012005C0E0001F96F000E000198
:10350000FA6F0001FC81010E0001FD6F0001FC8FCC
:1035100012002DECA0F0120000D03CEC8EF0120056
:103520000D012451010D5D0EF3240001F96F000E11
:10353000F4200001FA6F0001FC81010E0001FD6F13
:103540000001FC8F12000001FC8F0D012451010DC0
:103550005D0EF324D96E000EF420DA6E22CDDFFF6B
:103560001200000E2F6E020E2E6E000E306E000E38
:10357000316E000E336E000E326E38ECA6F0120083
:103580000D012151000AD8B4C4D7010AD8B4C5D757
:10359000020AD8B4C2D7060AD8B4A1D7030AD8B44D
:1035A000A4D7010AD8B4DDD70F0AD8B4A4D7010A2A
:1035B000D8B49ED7030AD8B4B3D7010AD8B4C3D7B6
:1035C000070A12001200E5C0D9FFE6C0DAFF000EBC
:1035D000DFBC010E116E040E0001E51B080E000198
:1035E000EF19D8A40FD00D0122517F0B0F01386FB6
:1035F0000F013851D8B402D0100E01D0040E0001D2
:10360000EF6F00D05604D8A43BD0000120EE02F0AA
:10361000E551D926E651DA22280EDE6E0D0EDD6E5A
:10362000DAEC9BF0020E5B18D8A40DD0E5C0D9FFF0
:10363000E6C0DAFF040EDF6EE5C0D9FFE6C0DAFFB0
:10364000000EDB8E12001150D8A40DD0E5C0D9FFBA
:10365000E6C0DAFF480EDF6EE5C0D9FFE6C0DAFF4C
:10366000000EDB8E1200E5C0D9FFE6C0DAFF080EBF
:10367000DF6EE5C0D9FFE6C0DAFF000EDB8E120078
:103680000001DFAF19D00001E2510001E311000198
:10369000E411D8B40ED020EEE2F001D80AD0050033
:1036A000FA6EDE50FD6EDE50FE6EDE50FF6EFA509A
:1036B00012000001DF9F00D0000E566E12001200B3
:1036C00062C06AF063C06BF060C068F061C069F00E
:1036D0000001685100016A5D0001695100016B59E8
:1036E000D8B045D00001645100016A250001666F21
:1036F0000001655100016B210001676F00016651F7
:103700000001685D0001675100016959D8B02FD0F0
:103710000001645100016A270001655100016B231B
:10372000000164510001682700016551000169230F
:1037300000D000016A07D8A06B076AC0D9FF6BC030
:10374000DAFF00016807D8A0690768C0E1FF69C017
:10375000E2FFDFCFE7FF00016407D8A065070001A3
:10376000645100016511D8B41200E3D712000001C2
:10377000645100016511D8B412006AC0D9FF6BC052
:10378000DAFF68C0E1FF69C0E2FFDFCFE7FF0001B9
:103790006A4B6B2B0001684B692B00016407D8A0B2
:1037A00065070001645100016511D8B41200E5D726
:1037B00012001200080E106E0001FE5112E1080EF8
:1037C0000001FD5DD8B00DD0FDC010F05B50D8A455
:1037D00002D0010E04D05B04D8A403D0020E5B6EAD
:1037E00000D010500001FD5F000EFE5B000120EED6
:1037F00001F0E551D926E651DA2210C0DFFF280E8C
:103800000101C16F0D0E0101C26F0001FCA120D0AA
:1038100043D01ED0F9C0F6FFFAC0F7FF000EF86ED5
:10382000C1C1D9FFC2C1DAFF0E0EF76403D0080090
:10383000F55005D0F6CFE9FFF7CFEAFFEF50DF6E86
:103840000001F94BFA2B0101C14BC22B100600D02D
:103850001050D8B41200DED712001ED0F9C0F6FF07
:10386000FAC0F7FF000EF86EC1C1D9FFC2C1DAFF7E
:103870000E0EF76403D00800F55005D0F6CFE9FF2F
:10388000F7CFEAFFEF50DF6E0001F94BFA2B010191
:10389000C14BC22B100600D01050D8B41200DED796
:1038A000120012000001726F030E0001F76528D0AC
:1038B000070E0001F76124D04F0E0001726520D081
:1038C000540E000172611CD0B00E0001722500017F
:1038D000686F0001696BFF0E6923000E00016B6FBA
:1038E000030E6A6F32ECABF0AB0E000168250001ED
:1038F0006E6FFF0E0001692100016F6F120000D092
:10390000000E0001636F0C0E626F72C060F0000168
:10391000616B5DEC9FF060C068F061C069F0000E03
:1039200000016B6F240E6A6F32ECABF0880E000161
:10393000706FF70E0001716F000168510001702770
:103940000001695100017123000E0001636F0C0E2C
:10395000626F72C060F00001616BACECA1F060C0FE
:1039600068F061C069F0000E00016B6F030E6A6FB2
:1039700032ECABF0000168510001702500016E6F60
:10398000000169510001712100016F6F12001200E6
:103990000001FC8F270E106E0F0E116E000E136EBD
:1039A000000E126E000E156E010E146E97ECABF049
:1039B000000E106E0D0E116E000E136E000E126EC4
:1039C000000E156E200E146E97ECABF0658C000E99
:1039D000366E010E366401D016D03650010DE90E58
:1039E000F324D96E000EF420DA6E000EDF6E36502E
:1039F000010DEB0EF324D96E000EF420DA6E000EEA
:103A0000DF6E362AE6D75D0E106E000E116E000EC8
:103A1000136E000E126E000E156E010E146E97ECF2
:103A2000ABF0659C080E0001E56F0D0E0001E66F1E
:103A3000000E4E6E0D0E4F6E4EC050F04FC051F046
:103A400022CD5CF05C50D8A404D0100E0001EF6FC2
:103A50001200000E2F6E010E2E6E5C0E306E000EE8
:103A6000316E000E336E010E326E38ECA6F0200E71
:103A70000001EF6F12001200000E00016A6F000ECD
:103A800000016B6F000E00016D6F070E00016D6588
:103A900001D011D000016D51010DEF0EF324D96E4C
:103AA000010EF420DA6E010EDF6402D000016A2BF1
:103AB00000016D2BEAD7000E00016D6F0B0E0001A7
:103AC0006D6501D011D000016D51010DD30EF324AD
:103AD000D96E010EF420DA6E010EDF6402D000010F
:103AE0006B2B00016D2BEAD7000E00016C6F010EED
:103AF00000016A6508D0010E00016B6504D0010E5B
:103B000000016C6F00D06CC069F0EF0E0001606FB7
:103B1000010E0001616F000E0001636F000E626F05
:103B2000000E0001656F080E646F4EECABF0D30E13
:103B30000001606F010E0001616F000E0001636FF4
:103B4000000E626F000E0001656F0C0E646F4EEC8C
:103B5000ABF00001695112001200000EC0B0010E5E
:103B60000001836F000183510001D8B403D0040029
:103B7000C09000D0010E02013F6F0001FF2B000139
:103B8000FF51800A700FD8A018D0000E0001606F9E
:103B9000F80E616F010E626F000E636F000E000180
:103BA000646FFC0E656F010E666F000E676FACEC04
:103BB000A3F0000E0001FF6F00D00001FF510001D3
:103BC000686F696B68BF6907000E00016B6F400E7C
:103BD0006A6F32ECABF0000168C07FF0000169C091
:103BE00080F0000E000180BFFF0E816F826F000E1B
:103BF00000017F2500016E6FF80E00018021000199
:103C00006F6F010E000181210001706F000E000135
:103C100082210001716F010E0001726F000E000120
:103C2000736F020E0001746FE0EC99F0000183B134
:103C300002D0C09001D0C08012000001646F00016A
:103C400060510001D8B408D000016451020DE50EA6
:103C5000F324D96E000E07D000016451020DBD0E91
:103C6000F324D96E010EF420DA6EDECF65F0DDCFDD
:103C700066F000D00001655100016611D8A407D09C
:103C8000000E0001606F000E0001616F1200000164
:103C900020EE02F06551D9266651DA2261C0DEFFBE
:103CA00062C0DDFF000120EE01F06551D9266651AA
:103CB000DA2263C0DFFF65C0D9FF66C0DAFF400EBD
:103CC000DF1665C0D9FF66C0DAFF000EDB8665C06F
:103CD000D9FF66C0DAFF000EDB8E000160510001E3
:103CE000D8B408D000016451020DE50EF324D96E5A
:103CF000000E07D000016451020DBD0EF324D96EF1
:103D0000010EF420DA6E040EDF1A00D065C060F0F8
:103D100066C061F0120012000101CA51D8A412005D
:103D2000010E0101CA6F0101CB51D8A41200010E8E
:103D30000101CB6F020E5618D8A416D0000120EE58
:103D400001F0E551D926E651DA22000EDF6EE5C01A
:103D5000D9FFE6C0DAFF480EDF6EE5C0D9FFE6C046
:103D6000DAFF000EDB8E12005604D8A41200000EFB
:103D70000101C76F20EE01F04E50D9264F50DA22D4
:103D8000080EDF6E20EE02F04E50D9264F50DA2298
:103D9000200EDE6E0D0EDD6E4EC0D9FF4FC0DAFF75
:103DA000040EDF6E4EC0D9FF4FC0DAFF000EDB8E6F
:103DB000010E0101C76F20EE01F05050D92651507D
:103DC000DA22080EDF6E20EE02F05050D926515054
:103DD000DA22200EDE6E0D0EDD6E50C0D9FF51C00E
:103DE000DAFF800EDF6E120012000001626F000128
:103DF000F551D8A43AD05DD038D000D0EDC060F0F5
:103E0000010E0001616F0001602B03D00001D8900A
:103E100061370001602FFAD700016151FF0A0001EC
:103E20006217EDC060F059C061F00001602B03D053
:103E30000001D89061370001602FFAD711D000D06F
:103E4000EDC060F0FD0E0001602759C061F0000177
:103E5000602B03D00001D89061370001602FFAD7A2
:103E6000000161510001621315D00001ED51000AFB
:103E7000D8B4C4D7010AD8B4C1D7030AD8B4BED7BE
:103E8000010AD8B4DDD7070AD8B4DAD7010AD8B402
:103E9000D7D700D0020E0001F819D8A40AD05AA230
:103EA00003D00001628100D05AAA03D000016285CC
:103EB00000D00001625112001200000E0001656F77
:103EC000000163AF09D00001626D631FD8B0632B9E
:103ED000010E0001656F00D0000161AF09D0000143
:103EE000606D611FD8B0612B010E0001651B00D011
:103EF000000E0001676F000E666F00016251000145
:103F00006311D8B431D0010E0001646F07D00001F5
:103F1000D890623763370001642B00D0000163BF83
:103F200002D0F5D700D00001D8906637673700017E
:103F300062510001605D0001635100016159D8A028
:103F40000BD0000162510001605F0001635100016C
:103F5000615B0001668100D00001D8906333623359
:103F60000001642FE0D700D0000165510001D8B4F2
:103F700006D00001666D671FD8B0672B00D066C001
:103F800060F067C061F0120012002D0E556E5EC029
:103F90003CF0FD0E3C16D8A457D05EC03CF0D89043
:103FA0003C323F0E3C163C50040D000EF3244E6E86
:103FB0000D0EF4204F6E4EC050F04FC051F0040E65
:103FC000501A4EC0D9FF4FC0DAFFDF30E8320F0B76
:103FD0000D0AD8A436D0000E3E6E070E3E6401D006
:103FE00023D020EE02F04E50D9264F50DA22DECFF9
:103FF0003CF0DDCF3DF03CC0D9FF3DC0DAFF3E5084
:10400000010D200EF324E16E0D0EF420E26EDFCFE1
:10401000E7FF20EE02F04E50D9264F50DA22DE2A7A
:10402000000EDD223E2AD9D720EE02F04E50D926CE
:104030004F50DA22200EDE6E0D0EDD6E44ECA4F041
:104040001200A6ECA7F012005E50FD0B040AD8A4E3
:104050001200E3EC9AF012001200000E0D01286F1E
:10406000000E0D01296F40D00001FC8F03D00D011F
:10407000288100D05204D8A443D00D01288340D019
:104080000001FC8F3DD00001FC8F0D0124BF0BD03F
:104090000D0124510F0B106E1050020DBD0EF324B4
:1040A000D96E010E0AD00D0124510F0B106E105065
:1040B000020DE50EF324D96E000EF420DA6EDECF89
:1040C00011F0DDCF12F000D011C0D9FF12C0DAFF1D
:1040D000DFAE16D011C0D9FF12C0DAFFDFA410D0B6
:1040E000010E0D01286F0CD00D0120511F0B000A8D
:1040F000D8B4BAD7010AD8B4C3D7030AD8B4C3D73F
:104100000001FCAF1200280E0001F96F0D0E000136
:10411000FA6F0001FC81020E0001FD6F1200120017
:10412000146E1050D8B407D01450020DE50EF324CD
:10413000D96E000E06D01450020DBD0EF324D96EB8
:10414000010EF420DA6EDECF15F0DDCF16F000D0D0
:1041500015501610D8A405D0000E106E000E116E6A
:10416000120020EE02F01550D9261650DA2211C0A6
:10417000DEFF12C0DDFF20EE01F01550D9261650EB
:10418000DA2213C0DFFF15C0D9FF16C0DAFF400ED8
:10419000DF1615C0D9FF16C0DAFF000EDB8615C08A
:1041A000D9FF16C0DAFF000EDB8E1050D8B407D04E
:1041B0001450020DE50EF324D96E000E06D01450F3
:1041C000020DBD0EF324D96E010EF420DA6E040E3A
:1041D000DF1A00D015C010F016C011F01200120046
:1041E0000001856F4FD09B8C200E0001846F2A0E3A
:1041F000E82EFED7842FFCD7F29CF29ED39E0F01AF
:1042000048691F0E0F01496F000E896E800E926E75
:10421000000E8A6E100E936E000E8B6EF00E946E72
:10422000200E8C6E110E956E000E8D6E000E966E29
:1042300000D0969EF18ED00E9216F80E9616100EA5
:104240009316310E951600D080EC90F05BECA3F045
:10425000CC0E8BECADF0010E0001616F380E606F7B
:104260003C0E15ECA5F01200130ED36E1200600E7A
:10427000D36E200E0001846F2A0EE82EFED7842F05
:10428000FCD7120000018551000AD8B4ACD7010A4E
:10429000D8B4EAD7030AD8A41200E9D71200830FD2
:1042A000830F830F830F830F830F810F810F810F84
:1042B000810F810F810F810F810F810F810F810F7E
:1042C000810F830F830F830F830F830F830F920F51
:1042D000920F920F920F920F920F960F960F960FCA
:1042E000960F960F920F920F920F920F920F920FBE
:1042F000920F920F920F920F960F960F960F10201B
:1043000040800408201002010408804020100804A6
:10431000201008040102010204081020804020102F
:1043200002014080010204080204088040200102CA
:1043300004081020010202040810200102040402F3
:1043400001201008040201020408200102048B0F5E
:104350008B0F8B0F01020400000E0001656F00013E
:1043600061AF09D00001606D611FD8B0612B010EF3
:104370000001656F00D0000163AF06D00001626DDF
:10438000631FD8B0632B00D000016251000163119C
:10439000D8B42BD0010E0001646F07D00001D89073
:1043A000623763370001642B00D0000163BF02D085
:1043B000F5D700D0000162510001605D000163513A
:1043C00000016159D8A009D0000162510001605F6D
:1043D000000163510001615B00D00001D89063339C
:1043E00062330001642FE6D700D00001655100015F
:1043F000D8B406D00001606D611FD8B0612B00D029
:1044000060C060F061C061F0120012002D6E4CD0EF
:104410009B8C200E2C6E2A0EE82EFED72C2EFCD75D
:10442000F29CF29ED39E0F0148691F0E0F01496F47
:10443000000E896E800E926E000E8A6E100E936EC4
:10444000000E8B6EF00E946E200E8C6E110E956E1B
:10445000000E8D6E000E966E00D0969EF18ED00EE0
:104460009216F80E9616100E9316310E951600D071
:10447000F6EC94F0D4ECA4F0CC0E9CECADF0010E74
:10448000116E380E106E3C0E74ECA7F01200130E75
:10449000D36E1200600ED36E200E2C6E2A0EE82E04
:1044A000FED72C2EFCD712002D50000AD8B4B0D75E
:1044B000010AD8B4ECD7030AD8A41200EBD7120033
:1044C00000016A6F6AC060F00001616B000E0001BC
:1044D000636F0C0E626F5DEC9FF000016051000194
:1044E0006B6F6AC060F00001616B000E0001636FCA
:1044F0000C0E626FACECA1F00001605100016C6F1A
:104500000101CEA12FD0060E00016C652BD0010E4B
:1045100000016B6527D0070E00016C5F020E0001E1
:104520006B5F00016B51050D570E0001686FF70EB0
:104530000001696FF35000016827F45000016923FE
:1045400000016C51010DF35000016827F450000187
:10455000692368C0F6FF69C0F7FF000EF86E080017
:10456000F5501200000E1200120003EE00F0FE0ED5
:10457000EE6AE806FDE102EE00F0700EEE6AE80673
:10458000FDE101EEB9F0460EEE6AE806FDE100EE4F
:10459000DCF0230EEE6AE806FDE100EE4EF0110EAF
:1045A000EE6AE806FDE1860EF66E5A0EF76E010E13
:1045B000F86E02EE70F010EE18F00900F5CFEEFF85
:1045C000E550E150FAE19E0EF66E420EF76E010ED6
:1045D000F86E01EE00F010EEB9F00900F5CFEEFF35
:1045E000E550E150FAE1410EF66E5B0EF76E010EFA
:1045F000F86E0900F5CFFFF0400EF66E5B0EF76E19
:10460000010EF86E0900F5CF5FF0000132EFA9F05E
:10461000000E0101C86F000E0101C96F020E56188D
:10462000D8A41FD020EE01F05050D9265150DA22E4
:10463000080EDF6E20EE02F05050D9265150DA22DB
:10464000280EDE6E0D0EDD6E50C0D9FF51C0DAFFB0
:10465000480EDF6E50C0D9FF51C0DAFF000EDB8E6E
:1046600012000001FD510D01265D0001FE510D01FA
:104670002759D8B005D026CDFDF027CDFEF000D0CB
:10468000DAEC9BF0000120EE02F0E551D926E6516C
:10469000DA22280EDE6E0D0EDD6EE5C0D9FFE6C013
:1046A000DAFF480EDF6EE5C0D9FFE6C0DAFF000E84
:1046B000DB8E12001200400E0001606F020E00013E
:1046C000616F000E0001636F0E0E626F000E00013D
:1046D000656F300E646F4EECABF0000E0001F26FB0
:1046E000DF0E0001606F010E0001616F000E00011E
:1046F000636F000E626F000E0001656F080E646F3D
:104700004EECABF0E70E0001606F010E0001616F2F
:10471000000E0001636F000E626F000E0001656FF6
:10472000020E646F4EECABF0E90E0001606F010EFB
:104730000001616F000E0001636F0E0E626F000ECC
:104740000001656F060E646F4EECABF0020E0001C7
:10475000F06F8DECA5F01200000E0001686F60C0D4
:1047600069F061C06AF062C06BF063C06CF02ED07B
:104770006BC0F8FF6AC0F7FF69C0F6FFA684A68881
:10478000F2AE04D0F29E010E0001686F550EA76EC6
:10479000AA0EA76EA682000168510001D8B402D00B
:1047A000F28E00D0000E000169250001696F040E31
:1047B00000016A2100016A6F000E00016B210001F7
:1047C0006B6F000E00016C2100016C6F00016451E1
:1047D0000001695D0001655100016A5900016651DF
:1047E00000016B590001675100016C59D8A0C0D776
:1047F0001200156E000E166E0D0E176E1050116E13
:10480000126AD890113612361550136E146AD89069
:1048100013361436D890133614361150132612500E
:104820001422D89013361436D890133614361350F9
:1048300016261450172216C0D9FF17C0DAFFDF9EC4
:104840001050D8A407D01550020DBD0EF324D96E18
:10485000010E06D01550020DE50EF324D96E000EA0
:10486000F420DA6E16C0DEFF17C0DDFF00D016C0E0
:10487000D9FF17C0DAFFDF9C20EE04F01650D926CE
:104880001750DA22DF8C1200000E5B6E000E546EA1
:10489000000E0101C86F000E0101C96F000E010179
:1048A000C76F000E566EE5C0D9FFE6C0DAFF7F0E77
:1048B000DF16040E0001E51BE5C0D9FFE6C0DAFFF4
:1048C0007F0EDF16040E0001E51B50C0D9FF51C05A
:1048D000DAFF7F0EDF16000E0001FC6F000E0001F4
:1048E000FE6F000EFD6F000E0001DF6F000E000175
:1048F000E16F000EE06F65EC9AF0000E2F6E030E74
:104900002E6E000E306E000E316E000E336E000EF5
:10491000326E38ECA6F059EC99F0120033D062C038
:10492000D9FF63C0DAFF60C0E1FF61C0E2FFDE5083
:10493000E618D8B420D062C0D9FF63C0DAFFDF50D8
:104940000001666F676B0001661F671F664B672B70
:1049500060C0D9FF61C0DAFFDF500001686F00015D
:104960006851000166250001606F000E000167219B
:104970000001616F12000001604B612B0001624B6E
:10498000632B00D000016407D8A0650700016429EB
:10499000C6E100016529D8A4C2D7000E0001616FED
:1049A000000E606F12001200400E106E020E116EAB
:1049B000000E136E0E0E126E000E156E300E146E7B
:1049C00097ECABF0000E0001F26FDF0E106E010EDF
:1049D000116E000E136E000E126E000E156E080E94
:1049E000146E97ECABF0E70E106E010E116E000E18
:1049F000136E000E126E000E156E020E146E97EC02
:104A0000ABF0E90E106E010E116E000E136E0E0E5D
:104A1000126E000E156E060E146E97ECABF0020EC1
:104A20000001F06FFFECA5F012000001626F000EB4
:104A3000AD6E000EAC6E000162A102D0AD8800D058
:104A4000000162A303D0AD8CAC8C00D0000162A544
:104A500002D0AD8E00D0000162A702D0AC8802D097
:104A6000AC8A00D0000162A902D0AD8400D0000160
:104A700062AB02D0AC8600D0000162AD02D09D8A4C
:104A800002D09D9A00D0000162AF02D09D8801D073
:104A90009D9860C0B0FF000161517F6EAD8AAC8E01
:104AA000120000016B6F26D0010E596E32D0000E3D
:104AB000596E000E5A6E2DD0000169510001D8B414
:104AC00028D0D7ECABF00009D8B423D0010E0101F7
:104AD000CC1B1FD068C06AF0220E00016A17D8B440
:104AE00018D0D7ECABF00009D8B413D0870E000172
:104AF0006B6F0FD000016B51270AD8B4EBD71E0A99
:104B0000D8B4DAD7A90AD8B4CFD7010AD8B4CFD746
:104B100000D000016B5112001200020ED7ECAAF077
:104B20000001F76F090E0001F76504D0000E0001C7
:104B3000F76F00D0040ED7ECAAF00001F46F0B0E53
:104B40000001F46504D0000E0001F46F00D0030EE4
:104B5000D7ECAAF00001F16F040E0001F16504D05A
:104B6000000E0001F16F00D0080ED7ECAAF0000192
:104B7000F86F020E0001F86504D0000E0001F86F16
:104B800000D027ECADF0BAECA8F01200000E000146
:104B9000636F5950D8B42FD060C0D9FF61C0DAFF1D
:104BA000DF500001626FDD0E00016217D8A423D030
:104BB000000120EE01F06051D9266151DA22DF5068
:104BC0000001626F070E00016217D8A414D0000123
:104BD000F551D8B410D00101CC51D8B409D0030E8E
:104BE0000001F76505D0060E0001F76504D000D07E
:104BF000010E0001636F0001635112001200020EEA
:104C000080ECABF00001F76F090E0001F76504D0EE
:104C1000000E0001F76F00D0040E80ECABF0000135
:104C2000F46F0B0E0001F46504D0000E0001F46F68
:104C300000D0030E80ECABF00001F16F040E000118
:104C4000F16504D0000E0001F16F00D0080E80EC79
:104C5000ABF00001F86F020E0001F86504D0000E01
:104C60000001F86F00D035ECADF00AECA9F01200AD
:104C70000DD0120098ECADF0120094ECADF01200E3
:104C800080ECA9F0120094EC93F012002EC034F0E6
:104C90002FC035F03550000AD8B404D07F0AD8A40C
:104CA00012001AD03450010AD8B4EAD7030AD8B493
:104CB0001200010AD8B4E7D7060AD8B41200770A5E
:104CC000D8B41200010AD8B41200070AD8B4D5D754
:104CD000010AD8A41200CED73450FF0A12001200E5
:104CE0000001616F27D00101B651FF0A0001606F1A
:104CF000B0C1D9FFB1C1DAFF00016051DF16120067
:104D00000101B751FF0A0001606FB2C1D9FFB3C101
:104D1000DAFF00016051DF1612000101B851FF0AED
:104D20000001606FB4C1D9FFB5C1DAFF0001605165
:104D3000DF16120000016151010AD8B4D4D7030A6A
:104D4000D8B4DED7010AD8A41200E7D7120060C099
:104D500066F061C067F01FD066C0F6FF67C0F7FF5E
:104D6000000EF86E0E0EF76403D00800F55005D063
:104D7000F6CFE9FFF7CFEAFFEF5000016219D8A4A0
:104D800006D066C060F067C061F0120004D0000178
:104D9000664B672B00D000016407D8A065070001AF
:104DA0006429DAE100016529D8A4D6D7000E0001F4
:104DB000606F000E0001616F120012006EC076F08D
:104DC0006FC077F070C078F071C079F0F8CF7CF0E8
:104DD000F7CF7BF0F6CF7AF078C0F8FF77C0F7FF17
:104DE00076C0F6FF0BD0090074C0D9FF75C0DAFF9A
:104DF000F5CFDFFF0001744B752B00D00001720767
:104E0000D8A0730700017229EEE100017329D8A42C
:104E1000EAD77CC0F8FF7BC0F7FF7AC0F6FF12002C
:104E200070C076F071C077F06EC074F06FC075F02E
:104E30001DD076C0F6FF77C0F7FF000EF86E74C085
:104E4000D9FF75C0DAFF0E0EF76403D00800F550E5
:104E500005D0F6CFE9FFF7CFEAFFEF50DF6E000194
:104E6000764B772B0001744B752B00D00001720735
:104E7000D8A0730700017229DCE100017329D8A4CE
:104E8000D8D712000001606F070E0001F46511D041
:104E9000E60E00016019D8A402D0900E1ED0E20EDA
:104EA00000016019D8A402D0910E17D0650E10D061
:104EB00017D0030E0001F46513D0E60E000160194F
:104EC000D8B4EBD7E20E00016019D8B4EDD7E30EE9
:104ED00000016019D8A404D0E20E0001606F00D078
:104EE0000001605112001200126E000EAD6E000E35
:104EF000AC6E12A002D0AD8800D012A203D0AD8C4F
:104F0000AC8C00D012A402D0AD8E00D012A602D07C
:104F1000AC8802D0AC8A00D012A802D0AD8400D0F8
:104F200012AA02D0AC8600D012AC02D09D8A02D068
:104F30009D9A00D012AE02D09D8801D09D9810C0DD
:104F4000B0FF11507F6EAD8AAC8E1200020E561863
:104F5000D8A403D0F4EC96F01200000E566E0101B6
:104F6000C751D8A41FD020EE01F05050D92651507F
:104F7000DA22080EDF6E20EE02F05050D926515092
:104F8000DA22200EDE6E0D0EDD6E50C0D9FF51C04C
:104F9000DAFF0C0EDF6E50C0D9FF51C0DAFF000EF1
:104FA000DB8E1200000E0101C76F12001200000E0E
:104FB0000001676F06D000016651A7ECA9F000015F
:104FC000672B00016751010D61C064F062C065F09C
:104FD000F35000016427F4500001652364C0F6FF1C
:104FE00065C0F7FF000EF86E0800F5CF66F000D040
:104FF000000163510001675DD8B0120000016651E5
:105000000001D8B41200D7D712001200F19E968E7C
:10501000EF0E9312CE0E951200F000F000F0010E8C
:105020000001626F8350FF0A0001606FCE0E000125
:105030006017D8A40DD08150FF0A0001606FEF0EF9
:1050400000016017D8A404D0000E0001626F00D0E8
:1050500062C061F0969EF18E100E9316310E951679
:10506000000161511200120016C01EF017C01FF09F
:1050700018C020F019C021F0F8CF24F0F7CF23F0AA
:10508000F6CF22F020C0F8FF1FC0F7FF1EC0F6FFCA
:105090000AD009001CC0D9FF1DC0DAFFF5CFDFFF21
:1050A0001C4A1D2A00D01A06D8A01B061A28F1E1B6
:1050B0001B28D8A4EED724C0F8FF23C0F7FF22C0D6
:1050C000F6FF120012C018F013C019F010C016F04D
:1050D00011C017F01BD018C0F6FF19C0F7FF000E63
:1050E000F86E16C0D9FF17C0DAFF0E0EF76403D0B2
:1050F0000800F55005D0F6CFE9FFF7CFEAFFEF50F3
:10510000DF6E184A192A164A172A00D01406D8A0AA
:1051100015061428E0E11528D8A4DDD712000001F7
:10512000636F63C0CEF100016351F5EC9EF00001A6
:10513000636FFE0EF66E1F0EF76E000EF86E09001E
:10514000030EF55E0900000EF55AD8B00FD001012C
:10515000D12B0101D151800A7C0FD8A004D0000EC0
:105160000101D16F03D00001639100D000016351B0
:1051700012001200010ED7ECAAF00001F56F050E27
:105180000001F56504D0000E0001F56F00D0050E9A
:10519000D7ECAAF00001ED6F060E0001ED6504D01A
:1051A000040E0001ED6F00D0060ED7ECAAF000014E
:1051B000F36F030E0001F3651200000E0001F36FA0
:1051C000120012000001606F18D0B0C1D9FFB1C148
:1051D000DAFF0101B651DF121200B2C1D9FFB3C12B
:1051E000DAFF0101B751DF121200B4C1D9FFB5C116
:1051F000DAFF0101B851DF12120000016051010A0B
:10520000D8B4E3D7030AD8B4E8D7010AD8A4120067
:10521000ECD71200010E80ECABF00001F56F050E2B
:105220000001F56504D0000E0001F56F00D0050EF9
:1052300080ECABF00001ED6F060E0001ED6504D0CF
:10524000040E0001ED6F00D0060E80ECABF0000103
:10525000F36F030E0001F3651200000E0001F36FFF
:1052600012001200000EF0ECA0F05AECADF084EC4D
:105270008BF028EC92F099ECAAF000D037ECAAF071
:10528000200E0001EF6101D0F9D765A208D006EC2D
:10529000A8F00009D8B4F2D7B8ECAAF0EFD7535071
:1052A000D8A4ECD701D0EAD747EC94F0E7D73FEF8A
:1052B00010F0000E0001656F06D000016651A7ECEA
:1052C000A9F00001652B00016551010D61C063F07B
:1052D00062C064F0F35000016327F45000016423BE
:1052E00063C0F6FF64C0F7FF000EF86E0800F5CF4C
:1052F00066F000D0000166510001D8A4DED712008C
:10530000000E0101B96F000E0101BA6F000E050118
:10531000086F1E0E186E010E79ECAAF0000E106ECA
:10532000080E116E050E126E010E136E010E90EC3A
:10533000A0F010C0BBF111C0BCF1170E17ECADF01E
:105340006DECADF010C0C3F111C0C4F1120000014A
:10535000606FFE0E0001F6610ED00001F651010DE6
:10536000000EF324D96E030EF420DA6E60C0DFFF66
:105370000001F62B00D0FE0E0001F66112000001C4
:10538000F651010D000EF324D96E030EF420DA6EEF
:10539000000EDF6E120012000001636F000163A1B6
:1053A00004D0010E7DECADF004D0010E84ECADF024
:1053B00000D0000163A304D0020E7DECADF004D058
:1053C000020E84ECADF000D0000163A504D0030E02
:1053D0007DECADF01200030E84ECADF01200120073
:1053E0000F0126A11FD04EC0D9FF4FC0DAFF800E9B
:1053F000DE18D8A415D0E5C0D9FFE6C0DAFF840EC8
:10540000DE18D8A40DD04EC0D9FF4FC0DAFF0C0E65
:10541000DF6E4EC0D9FF4FC0DAFF000EDB8E00D02A
:105420000F012691629A12000101D0510001F65D30
:10543000D8B016D00001F651010D000EF324D96E3C
:10544000030EF420DA6EDF500001606F0001F62BCE
:10545000000160510001D8A4120002D0120000D057
:10546000000E0101D06FD0C1F6F01200120065A24B
:1054700018D0010E84ECADF0020E84ECADF0030EFA
:1054800084ECADF012000DD076ECADF01200010E00
:105490007DECADF0020E7DECADF0030E7DECADF0D9
:1054A00012000001EF51200AD8B4EED7F0D7120055
:1054B0000001876F02013E510A0D000E0001856F49
:1054C000020E0001866FF35000018527F4500001A1
:1054D000862300018751010DF35000018525D96E07
:1054E000F45000018621DA6E84C0DFFFADEC9DF040
:1054F00012001B6E18A406D0000E106E1B50F9ECA3
:10550000A3F000D018A206D0010E106E1B50F9ECCB
:10551000A3F000D01B50010D260EF324196E0F0EC0
:10552000F4201A6E19C0D9FF1AC0DAFF18C0DFFFC5
:1055300012000001EF51D8A41200000E656E000E9B
:105540000F01366F160E0F01396F9F0E0F01376F67
:105550007B0E0F01366FD08EA288A088F28E01D00C
:10556000658665A6FDD7010E0001EF6F12001200DF
:105570005250D8B412005350D8B41200A09890ECF6
:10558000ADF065922F0E0001866FC00EE82EFED79B
:10559000862FFCD76584200E0001866F2A0EE82E28
:1055A000FED7862FFCD76594A08812001200000158
:1055B000626F02013E510A0D000E0001606F020E83
:1055C0000001616FF35000016027F4500001612376
:1055D00000016251010DF35000016025D96EF450B5
:1055E00000016121DA6EDF5012001200000E536ECE
:1055F000000E2F6E740E2E6E000E306E000E316E89
:10560000000E336E000E326E38ECA6F065920F017C
:10561000369562A807D00F0136A904D0629802D04F
:10562000629400D062B4FCD7120000016051000106
:105630006111D8A402D0270E1200000160510001B0
:105640006111D8B40CD00001615109E10A0E0001CA
:10565000605DD8B004D0000160511D0F12002C0E07
:10566000120012000001685100016A03F3CF6CF0D0
:10567000F4CF6DF00001685100016B03F35000019D
:105680006D270001695100016A03F35000016D2785
:105690006CC068F06DC069F01200120060C066F066
:1056A00061C067F00AD066C0D9FF67C0DAFF62C088
:1056B000DFFF0001664B672B00D000016407D8A014
:1056C000650700016429EFE100016529D8A4EBD743
:1056D0001200280E0001DC6F0D0E0001DD6F000EC0
:1056E0000001E16F080EE06FFA0E0001E26FF70EA5
:1056F0000001E36F010E0001E46F0001DF8F120073
:10570000126E02013E510A0D000E106E020E116E55
:10571000F3501026F45011221250010DF3501024B2
:10572000D96EF4501120DA6EDF501200120010C052
:1057300016F011C017F009D016C0D9FF17C0DAFF54
:1057400012C0DFFF164A172A00D01406D8A015068B
:105750001428F2E11528D8A4EFD712000F013685DE
:1057600062986582010E536E000E2F6E750E2E6EBE
:10577000000E306E000E316E000E336E000E326E73
:1057800038ECA6F012000101D0510001F65DD8B04E
:105790000BD00001F651010D000EF324D96E030E5B
:1057A000F420DA6EDF501200000E12001200010E1B
:1057B0000001606F030E0001EE19D8B408D0040E8A
:1057C0000001EE19D8B403D0000E0001606F000193
:1057D00060511200120010501202F3CF14F0F4CFF7
:1057E00015F010501302F350152611501202F35009
:1057F000152614C010F015C011F01200120000019F
:10580000F82B020E0001F86504D0000E0001F86FBD
:1058100000D0F8C084F0080E58ECAAF08FECACF081
:1058200012000001F72B090E0001F76504D0000EED
:105830000001F76F00D0F7C084F0020E58ECAAF018
:10584000A0ECACF012000001F42B0B0E0001F4658B
:1058500004D0000E0001F46F00D0F4C084F0040EF8
:1058600058ECAAF0B1ECACF012000001ED2B060EE2
:105870000001ED6504D0000E0001ED6F00D0EDC019
:1058800084F0050E58ECAAF0C2ECACF01200000156
:10589000F52B050E0001F56504D0000E0001F56F33
:1058A00000D0F5C084F0010E58ECAAF0D3ECACF0B7
:1058B00012000001F32B030E0001F36504D0000E6B
:1058C0000001F36F00D0F3C084F0060E58ECAAF08C
:1058D000E4ECACF012000001F12B040E0001F165C4
:1058E00004D0000E0001F16F00D0F1C084F0030E6F
:1058F00058ECAAF0F5ECACF012000001EE2B040E0F
:105900000001EE6504D0000E0001EE6F00D0EEC085
:1059100084F0000E58ECAAF006ECADF01200000185
:10592000F851040DB70EF3240001616FFF0EF4204F
:105930000001626F040E0001636FD7ECA7F0120044
:105940000001F751050D8A0EF3240001616FFD0E71
:10595000F4200001626F050E0001636FD7ECA7F021
:1059600012000001F451050D1A0EF3240001616FBD
:10597000FD0EF4200001626F050E0001636FD7EC8D
:10598000A7F012000001ED51040D130EF3240001E5
:10599000616FFF0EF4200001626F040E0001636F5F
:1059A000D7ECA7F012000001F551060DA90EF32463
:1059B0000001616FFE0EF4200001626F060E00010F
:1059C000636FD7ECA7F012000001F351050D760EBE
:1059D000F3240001616FFF0EF4200001626F050ED9
:1059E0000001636FD7ECA7F012000001F151040D24
:1059F000620EF3240001616FFF0EF4200001626F5C
:105A0000040E0001636FD7ECA7F012000001EE5105
:105A1000050D490EF3240001616FFF0EF420000113
:105A2000626F050E0001636FD7ECA7F01200106ED5
:105A300010507F0BD56E000ED76E000ED66EF2940E
:105A400010AE02D0F28A01D0F29AD58E1200000E6A
:105A5000D7ECAAF00001EE6F040E0001EE65120013
:105A6000000E0001EE6F12001200000E80ECABF091
:105A70000001EE6F040E0001EE651200000E000141
:105A8000EE6F12001200830F830F810F810F810FC1
:105A9000810F830F830F830F810F810F810F00010F
:105AA000606F010E0001F66F60C0D0F1030100517C
:105AB00012001200010E7DECADF0020E7DECADF097
:105AC000030E7DECADF01200D6CF62F0D7CF63F0BD
:105AD00062C060F063C061F01200D6CF12F0D7CF81
:105AE00013F012C010F013C011F01200050108519C
:105AF0008FECA8F0CCECA9F012000001616F00015E
:105B00006151E2ECA8F012000001626F00016251E5
:105B100070ECA6F012000001606F60C07EFF120002
:105B2000020EF0ECA0F01200020E06ECA2F0120041
:105B3000010E06ECA2F01200106E10C07EFF1200E3
:025B400001FF63
:10F7F800080128CD08F512000000000000000000F4
:10F8080000000000000000000000000000000000F0
:10F8180000000000000000000000000000000000E0
:10F8280000000000000000000000000000000000D0
:10F8380000000000000000000000000000000000C0
:08FFF800AEF70DF261FA81F988
:00000001FF
